:020000040800F2
:1000000000000824051E00088D1A00088F1A000839
:10001000911A0008931A0008951A000800000000C1
:10002000000000000000000000000000971A000817
:10003000991A0008000000009B1A00089D1A000889
:10004000551E0008551E0008551E0008551E0008C4
:10005000551E0008551E0008551E0008551E0008B4
:10006000A51A0008551E0008B11A0008551E000800
:10007000551E0008551E0008551E0008551E000894
:10008000551E0008551E0008551E0008551E000884
:10009000551E0008551E0008551E0008551E000874
:1000A000551E0008551E0008551E0008551E000864
:1000B000C91A0008551E0008551E0008551E0008E4
:1000C000551E0008551E0008551E0008551E000844
:1000D000551E0008D91A0008551E0008551E0008B4
:1000E000551E0008551E000800000000551E00089F
:1000F000551E0008551E0008551E0008551E000814
:10010000551E0008551E0008551E0008551E000803
:10011000551E0008551E0008551E0008551E0008F3
:10012000551E0008551E0008551E0008551E0008E3
:10013000551E0008551E0008551E0008551E0008D3
:1001400000000000000000000000000000000000AF
:10015000551E0008551E0008551E0008551E0008B3
:10016000551E0008551E0008551E0008551E0008A3
:10017000551E0008551E0008551E0008551E000893
:10018000551E0008551E0008551E0008551E000883
:10019000551E0008551E0008551E0008551E000873
:1001A000551E0008551E0008551E0008551E000863
:1001B000551E0008551E0008551E0008551E000853
:1001C000551E0008551E0008551E0008551E000843
:1001D000551E0008551E0008551E0008551E000833
:1001E000551E0008551E0008551E0008551E000823
:1001F000551E0008551E0008551E0008551E000813
:10020000551E0008551E0008551E0008551E000802
:10021000551E0008551E0008551E0008551E0008F2
:10022000551E0008551E0008551E0008000000005D
:10023000551E0008551E000800000000551E00084D
:10024000551E0008551E0008551E0008551E0008C2
:10025000551E0008551E0008551E0008551E0008B2
:10026000551E0008551E0008551E0008551E0008A2
:10027000551E0008551E0008551E0008000000000D
:10028000551E0008551E0008551E000800000000FD
:0802900000000000551E0008EB
:1002C00010B5054C237833B9044B13B10448AFF390
:1002D00000800123237010BDC0090024000000002D
:1002E00050BB000808B5034B1BB103490348AFF3EB
:1002F000008008BD00000000C409002450BB0008B5
:1003000080F0004002E000BF81F0004142001FBFCA
:100310005FEA410392EA030F7FEA226C7FEA236CD3
:100320006AD04FEA1262D2EB1363C1BFD2184140C8
:1003300048404140B8BF5B42192B88BF704710F05E
:10034000004F40F4000020F07F4018BF404211F001
:10035000004F41F4000121F07F4118BF494292EA69
:10036000030F3FD0A2F1010241FA03FC10EB0C0095
:10037000C3F1200301FA03F100F0004302D5494222
:1003800060EB4000B0F5000F13D3B0F1807F06D3CF
:1003900040084FEA310102F10102FE2A51D2B1F1C7
:1003A000004F40EBC25008BF20F0010040EA0300BC
:1003B0007047490040EB0000013A28BFB0F5000F3C
:1003C000EDD2B0FA80FCACF1080CB2EB0C0200FAF2
:1003D0000CF0AABF00EBC25052421843BCBFD04041
:1003E0001843704792F0000F81F4000106BF80F4BB
:1003F00000000132013BB5E74FEA41037FEA226C7E
:1004000018BF7FEA236C21D092EA030F04D092F048
:10041000000F08BF0846704790EA010F1CBF00207C
:10042000704712F07F4F04D1400028BF40F00040D9
:10043000704712F100723CBF00F50000704700F0F9
:10044000004343F0FE4040F4000070477FEA226220
:1004500016BF08467FEA23630146420206BF5FEAF1
:10046000412390EA010F40F4800070474FF00003F1
:1004700004E000BF10F0004348BF40425FEA000CB8
:1004800008BF704743F0964301464FF000001CE060
:1004900050EA010208BF70474FF000030AE000BFB6
:1004A00050EA010208BF704711F0004302D54042F4
:1004B00061EB41015FEA010C02BF84460146002066
:1004C00043F0B64308BFA3F18053A3F50003BCFA81
:1004D0008CF2083AA3EBC25310DB01FA02FC63442E
:1004E00000FA02FCC2F12002BCF1004F20FA02F235
:1004F00043EB020008BF20F00100704702F1200228
:1005000001FA02FCC2F1200250EA4C0021FA02F288
:1005100043EB020008BF20EADC7070474FF0FF0C8D
:100520001CEAD0521EBF1CEAD15392EA0C0F93EA88
:100530000C0F6FD01A4480EA010C400218BF5FEA2A
:1005400041211ED04FF0006343EA501043EA51119D
:10055000A0FB01310CF00040B1F5000F3EBF490097
:1005600041EAD3715B0040EA010062F17F02FD2A9B
:100570001DD8B3F1004F40EBC25008BF20F001007E
:10058000704790F0000F0CF0004C08BF49024CEA95
:10059000502040EA51207F3AC2BFD2F1FF0340EA27
:1005A000C250704740F400004FF00003013A5DDC98
:1005B00012F1190FDCBF00F000407047C2F10002D9
:1005C000410021FA02F1C2F1200200FA02FC5FEAC6
:1005D000310040F1000053EA4C0308BF20EADC7010
:1005E000704792F0000F00F0004C02BF400010F482
:1005F000000F013AF9D040EA0C0093F0000F01F02F
:10060000004C02BF490011F4000F013BF9D041EA50
:100610000C018FE70CEAD15392EA0C0F18BF93EA52
:100620000C0F0AD030F0004C18BF31F0004CD8D17C
:1006300080EA010000F00040704790F0000F17BF03
:1006400090F0004F084691F0000F91F0004F14D049
:1006500092EA0C0F01D142020FD193EA0C0F03D1A1
:100660004B0218BF084608D180EA010000F00040A4
:1006700040F0FE4040F40000704740F0FE4040F47F
:10068000400070474FF0FF0C1CEAD0521EBF1CEA1E
:10069000D15392EA0C0F93EA0C0F69D0A2EB03023C
:1006A00080EA010C49024FEA402037D04FF08053D6
:1006B00043EA111143EA10130CF000408B4238BF9B
:1006C0005B0042F17D024FF4000C8B4224BF5B1AA9
:1006D00040EA0C00B3EB510F24BFA3EB510340EAF7
:1006E0005C00B3EB910F24BFA3EB910340EA9C00A5
:1006F000B3EBD10F24BFA3EBD10340EADC001B0115
:1007000018BF5FEA1C1CE0D1FD2A3FF650AF8B42B8
:1007100040EBC25008BF20F0010070470CF0004CC5
:100720004CEA50207F32C2BFD2F1FF0340EAC250F0
:10073000704740F400004FF00003013A37E792F0B1
:10074000000F00F0004C02BF400010F4000F013A0F
:10075000F9D040EA0C0093F0000F01F0004C02BF0A
:10076000490011F4000F013BF9D041EA0C0195E773
:100770000CEAD15392EA0C0F08D142027FF47DAF0C
:1007800093EA0C0F7FF470AF084676E793EA0C0FFC
:1007900004D14B023FF44CAF08466EE730F0004CFA
:1007A00018BF31F0004CCAD130F000427FF45CAF8A
:1007B00031F000437FF43CAF5FE700BF42000ED250
:1007C000B2F1FE4F0BD34FF09E03B3EB126209D48C
:1007D0004FEA002343F0004323FA02F070474FF042
:1007E0000000704712F1610F01D1420202D14FF0B7
:1007F000FF3070474FF00000704700BF53B94AB94F
:10080000002908BF00281CBF4FF0FF314FF0FF3018
:1008100000F074B9ADF1080C6DE904CE00F006F8F3
:10082000DDF804E0DDE9022304B070472DE9F0476C
:10083000089E0D4604468846002B4DD18A429446B8
:1008400068D9B2FA82F252B101FA02F3C2F1200180
:1008500020FA01F10CFA02FC41EA030894404FEA45
:100860001C45210CB8FBF5FE1FFA8CF705FB1E8317
:1008700041EA03430EFB07F199420BD91CEB03033A
:100880000EF1FF3080F01E81994240F21B81AEF1E3
:10089000020E63445B1AA4B2B3FBF5F005FB103300
:1008A00044EA034400FB07F7A7420AD91CEB0404FF
:1008B00000F1FF3380F00881A74240F205816444D3
:1008C0000238E41B40EA0E4000211EB1D440002350
:1008D000C6E90043BDE8F0878B4208D9002E00F03E
:1008E000EE800021C6E900050846BDE8F087B3FAAE
:1008F00083F100294AD1AB4202D3824200F2F9804F
:10090000841A65EB030301209846002EE2D0C6E965
:100910000048DFE702B9FFDEB2FA82F2002A40F0B7
:100920009180A1EB0C054FEA1C471FFA8CFE0121B8
:10093000B5FBF7F307FB1350250C45EA00450EFB0A
:1009400003F0A84208D91CEB050503F1FF3802D2D9
:10095000A84200F2CB8043462D1AA4B2B5FBF7F0B3
:1009600007FB105544EA05440EFB00FEA64508D9D6
:100970001CEB040400F1FF3502D2A64500F2BB8057
:100980002846A4EB0E0440EA03409EE7C1F120078D
:100990008B4022FA07FC4CEA030C20FA07F405FA14
:1009A00001F31C43FD404FEA1C4900FA01F3B5FB7B
:1009B000F9F8200C1FFA8CFE09FB185540EA054592
:1009C00008FB0EF0A84202FA01F20BD91CEB050558
:1009D00008F1FF3A80F08880A84240F28580A8F1B3
:1009E000020865442D1AA4B2B5FBF9F009FB1055B5
:1009F00044EA054500FB0EFEAE4508D91CEB050593
:100A000000F1FF346CD2AE456AD90238654440EA41
:100A10000840A0FB0294A5EB0E05A542C846A646D9
:100A200056D353D05EB1B3EB080265EB0E0505FA61
:100A300007F722FA01F3CD401F43C6E900750021F4
:100A4000BDE8F087C2F1200320FA03F10CFA02FCA2
:100A500025FA03F395400D434FEA1C471FFA8CFE1D
:100A6000B3FBF7F107FB11302B0C43EA004301FB0A
:100A70000EF0984204FA02F408D91CEB030301F1CA
:100A8000FF382FD298422DD9023963441B1AADB2D8
:100A9000B3FBF7F007FB103345EA034500FB0EF309
:100AA000AB4208D91CEB050500F1FF3816D2AB426A
:100AB00014D902386544ED1A40EA014138E731465D
:100AC000304607E78646E5E61846FAE64B45A9D2E2
:100AD000B9EB020864EB0C0E0138A3E74046EAE7E5
:100AE000204694E74146D1E7D0467BE7023B654488
:100AF00032E7084609E76444023842E7704700BF1E
:100B000001F0FF01102A2BDB10F0070F08D010F8BE
:100B1000013B013A8B422DD010F0070F42B3F6D1C2
:100B2000F0B441EA012141EA014122F007047FF0DB
:100B300000070023F0E80256083C85EA010586EA32
:100B4000010685FA47F5A3FA87F586FA47F6A5FA6E
:100B500087F68EB9EED1F0BC01F0FF0102F007027A
:100B600032B110F8013B013A83EA010313B1F8D125
:100B70000020704701387047002D06BF3546033806
:100B8000073815F0010F07D1013015F4807F02BF3F
:100B9000013015F4C03F0130F0BC0138704700BF90
:100BA000844641EA000313F003036DD1403A41D378
:100BB00051F8043B40F8043B51F8043B40F8043B37
:100BC00051F8043B40F8043B51F8043B40F8043B27
:100BD00051F8043B40F8043B51F8043B40F8043B17
:100BE00051F8043B40F8043B51F8043B40F8043B07
:100BF00051F8043B40F8043B51F8043B40F8043BF7
:100C000051F8043B40F8043B51F8043B40F8043BE6
:100C100051F8043B40F8043B51F8043B40F8043BD6
:100C200051F8043B40F8043B51F8043B40F8043BC6
:100C3000403ABDD2303211D351F8043B40F8043B66
:100C400051F8043B40F8043B51F8043B40F8043BA6
:100C500051F8043B40F8043B103AEDD20C3205D376
:100C600051F8043B40F8043B043AF9D2043208D06E
:100C7000D2071CBF11F8013B00F8013B01D30B88E0
:100C800003806046704700BF082A13D38B078DD0BE
:100C900010F003038AD0C3F10403D21ADB071CBF90
:100CA00011F8013B00F8013B80D331F8023B20F8FA
:100CB000023B7BE7043AD9D3013A11F8013B00F833
:100CC000013BF9D20B7803704B7843708B788370BB
:100CD00060467047000000000000000000000000B7
:100CE0000000000000000000000000000000000004
:100CF00000000000000000000000000000000000F4
:100D000090F800F06DE9024520F007016FF0000C4B
:100D100010F0070491F820F040F049804FF00004F3
:100D20006FF00700D1E9002391F840F000F10800CE
:100D300082FA4CF2A4FA8CF283FA4CF3A2FA8CF306
:100D40004BBBD1E9022382FA4CF200F10800A4FA6D
:100D50008CF283FA4CF3A2FA8CF3E3B9D1E90423C1
:100D600082FA4CF200F10800A4FA8CF283FA4CF3F8
:100D7000A2FA8CF37BB9D1E9062301F1200182FAB2
:100D80004CF200F10800A4FA8CF283FA4CF3A2FAB8
:100D90008CF3002BC6D0002A04BF04301A4612BAC6
:100DA000B2FA82F2FDE8024500EBD2007047D1E9C9
:100DB000002304F00305C4F100004FEAC50514F058
:100DC000040F91F840F00CFA05F562EA05021CBF29
:100DD00063EA050362464FF00004A9E781F0004191
:100DE00002E000BF83F0004330B54FEA41044FEA10
:100DF000430594EA050F08BF90EA020F1FBF54EAAB
:100E0000000C55EA020C7FEA645C7FEA655C00F046
:100E1000E2804FEA5454D4EB5555B8BF6D420CDD17
:100E20002C4480EA020281EA030382EA000083EA9A
:100E3000010180EA020281EA0303362D88BF30BD3A
:100E400011F0004F4FEA01314FF4801C4CEA113190
:100E500002D0404261EB410113F0004F4FEA0333EF
:100E60004CEA133302D0524263EB430394EA050F7A
:100E700000F0A780A4F10104D5F1200E0DDB02FAE9
:100E80000EFC22FA05F2801841F1000103FA0EF27D
:100E9000801843FA05F359410EE0A5F120050EF143
:100EA000200E012A03FA0EFC28BF4CF0020C43FA74
:100EB00005F3C01851EBE37101F0004507D54FF081
:100EC000000EDCF1000C7EEB00006EEB0101B1F5D1
:100ED000801F1BD3B1F5001F0CD349085FEA300017
:100EE0004FEA3C0C04F101044FEA445212F5800F22
:100EF00080F09A80BCF1004F08BF5FEA500C50F1BF
:100F0000000041EB045141EA050130BD5FEA4C0CA1
:100F1000404141EB0101013C28BFB1F5801FE9D2FE
:100F200091F0000F04BF01460020B1FA81F308BF21
:100F30002033A3F10B03B3F120020CDA0C3208DDED
:100F400002F1140CC2F10C0201FA0CF021FA02F1C8
:100F50000CE002F11402D8BFC2F1200C01FA02F138
:100F600020FA0CFCDCBF41EA0C019040E41AA2BF5D
:100F700001EB0451294330BD6FEA04041F3C1CDA25
:100F80000C340EDC04F11404C4F1200220FA04F045
:100F900001FA02F340EA030021FA04F345EA0301EF
:100FA00030BDC4F10C04C4F1200220FA02F001FAB1
:100FB00004F340EA0300294630BD21FA04F0294633
:100FC00030BD94F0000F83F4801306BF81F48011CC
:100FD0000134013D4EE77FEA645C18BF7FEA655C3F
:100FE00029D094EA050F08BF90EA020F05D054EA11
:100FF000000C04BF1946104630BD91EA030F1EBF16
:101000000021002030BD5FEA545C05D14000494119
:1010100028BF41F0004130BD14F580043CBF01F50C
:10102000801130BD01F0004545F0FE4141F47001F2
:101030004FF0000030BD7FEA645C1ABF19461046CD
:101040007FEA655C1CBF0B46024650EA013406BFCE
:1010500052EA033591EA030F41F4002130BD00BF8D
:1010600090F0000F04BF0021704730B54FF480644A
:1010700004F132044FF000054FF0000150E700BFCB
:1010800090F0000F04BF0021704730B54FF480642A
:1010900004F1320410F0004548BF40424FF0000117
:1010A0003EE700BF42004FEAE2014FEA31014FEA5A
:1010B00002701FBF12F07F4393F07F4F81F06051A9
:1010C000704732F07F4208BF704793F07F4F04BFF4
:1010D00041F40021704730B54FF4607401F00045D1
:1010E00021F000411CE700BF50EA010208BF704731
:1010F00030B54FF000050AE050EA010208BF704722
:1011000030B511F0004502D5404261EB41014FF48A
:10111000806404F132045FEA915C3FF4D8AE4FF092
:1011200003025FEADC0C18BF03325FEADC0C18BF75
:10113000033202EBDC02C2F1200300FA03FC20FAC6
:1011400002F001FA03FE40EA0E0021FA02F1144413
:10115000BDE600BF70B54FF0FF0C4CF4E06C1CEA2C
:1011600011541DBF1CEA135594EA0C0F95EA0C0F9D
:1011700000F0DEF82C4481EA030621EA4C5123EA10
:101180004C5350EA013518BF52EA033541F480113F
:1011900043F4801338D0A0FB02CE4FF00005E1FBF2
:1011A00002E506F00042E0FB03E54FF00006E1FB3C
:1011B00003569CF0000F18BF4EF0010EA4F1FF047F
:1011C000B6F5007F64F5407404D25FEA4E0E6D41BF
:1011D00046EB060642EAC62141EA55514FEAC520D0
:1011E00040EA5E504FEACE2EB4F1FD0C88BFBCF54C
:1011F000E06F1ED8BEF1004F08BF5FEA500E50F1FD
:10120000000041EB045170BD06F0004646EA0101C2
:1012100040EA020081EA0301B4EB5C04C2BFD4EBF4
:101220000C0541EA045170BD41F480114FF0000EED
:10123000013C00F3AB8014F1360FDEBF002001F05B
:10124000004170BDC4F10004203C35DA0C341BDCD5
:1012500004F11404C4F1200500FA05F320FA04F0A7
:1012600001FA05F240EA020001F0004221F00041DB
:1012700010EBD37021FA04F642EB06015EEA430E4E
:1012800008BF20EAD37070BDC4F10C04C4F120057E
:1012900000FA04F320FA05F001FA04F240EA020031
:1012A00001F0004110EBD37041F100015EEA430E02
:1012B00008BF20EAD37070BDC4F1200500FA05F222
:1012C0004EEA020E20FA04F301FA05F243EA0203A1
:1012D00021FA04F001F0004121FA04F220EA0200B0
:1012E00000EBD3705EEA430E08BF20EAD37070BDF6
:1012F00094F0000F0FD101F00046400041EB0101D6
:1013000011F4801F08BF013CF7D041EA060195F0B7
:10131000000F18BF704703F00046520043EB030371
:1013200013F4801F08BF013DF7D043EA060370475E
:1013300094EA0C0F0CEA135518BF95EA0C0F0CD069
:1013400050EA410618BF52EA4306D1D181EA0301AF
:1013500001F000414FF0000070BD50EA410606BFA9
:101360001046194652EA430619D094EA0C0F02D1EE
:1013700050EA013613D195EA0C0F05D152EA033633
:101380001CBF104619460AD181EA030101F0004151
:1013900041F0FE4141F470014FF0000070BD41F09A
:1013A000FE4141F4780170BD70B54FF0FF0C4CF474
:1013B000E06C1CEA11541DBF1CEA135594EA0C0F93
:1013C00095EA0C0F00F0A7F8A4EB050481EA030EE0
:1013D00052EA03354FEA013100F088804FEA0333C7
:1013E0004FF0805545EA131343EA12634FEA022295
:1013F00045EA111545EA10654FEA00260EF0004156
:101400009D4208BF964244F1FD0404F5407402D2A7
:101410005B084FEA3202B61A65EB03055B084FEA38
:1014200032024FF480104FF4002CB6EB020E75EB35
:10143000030E22BFB61A754640EA0C005B084FEA5D
:101440003202B6EB020E75EB030E22BFB61A7546DA
:1014500040EA5C005B084FEA3202B6EB020E75EB25
:10146000030E22BFB61A754640EA9C005B084FEA9D
:101470003202B6EB020E75EB030E22BFB61A7546AA
:1014800040EADC0055EA060E18D04FEA051545EA99
:1014900016754FEA06164FEAC30343EA52734FEA42
:1014A000C2025FEA1C1CC0D111F4801F0BD141EABB
:1014B00000014FF000004FF0004CB6E711F4801F20
:1014C00004BF01430020B4F1FD0C88BFBCF5E06F00
:1014D0003FF6AFAEB5EB030C04BFB6EB020C5FEA10
:1014E000500C50F1000041EB045170BD0EF0004E65
:1014F0004EEA113114EB5C04C2BFD4EB0C0541EA97
:10150000045170BD41F480114FF0000E013C90E693
:1015100045EA060E8DE60CEA135594EA0C0F08BF57
:1015200095EA0C0F3FF43BAF94EA0C0F0AD150EA56
:1015300001347FF434AF95EA0C0F7FF425AF1046E9
:1015400019462CE795EA0C0F06D152EA03353FF411
:10155000FDAE1046194622E750EA410618BF52EA8E
:1015600043067FF4C5AE50EA41047FF40DAF52EA62
:1015700043057FF4EBAE12E74FF0FF3C06E000BFFF
:101580004FF0010C02E000BF4FF0010C4DF804CD0C
:101590004FEA410C7FEA6C5C4FEA430C18BF7FEACC
:1015A0006C5C1BD001B050EA410C0CBF52EA430CFA
:1015B00091EA030F02BF90EA020F0020704710F17A
:1015C000000F91EA030F58BF994208BF90422CBF09
:1015D000D8176FEAE37040F0010070474FEA410C02
:1015E0007FEA6C5C02D150EA013C07D14FEA430C20
:1015F0007FEA6C5CD6D152EA033CD3D05DF8040B91
:10160000704700BF8446104662468C4619466346C2
:1016100000E000BF01B5FFF7B7FF002848BF10F199
:10162000000F01BD4DF808EDFFF7F4FF0CBF0120DE
:1016300000205DF808FB00BF4DF808EDFFF7EAFF5A
:1016400034BF012000205DF808FB00BF4DF808ED15
:10165000FFF7E0FF94BF012000205DF808FB00BF0A
:101660004DF808EDFFF7CEFF94BF012000205DF894
:1016700008FB00BF4DF808EDFFF7C4FF34BF0120A1
:1016800000205DF808FB00BF4FEA410C7FEA6C5C6C
:1016900002D150EA013C0AD14FEA430C7FEA6C5C6C
:1016A00002D152EA033C02D14FF0000070474FF0E4
:1016B000010070474FEA410212F5001215D211D510
:1016C0006FF47873B3EB625212D94FEAC12343F03F
:1016D000004343EA505311F0004F23FA02F018BFC1
:1016E000404270474FF00000704750EA013005D18A
:1016F00011F0004008BF6FF0004070474FF000004D
:10170000704700BF10B588B000240394049405947A
:1017100006940794194BD3F8E02042F08002C3F8F6
:10172000E020D3F8E02002F080020192019AD3F881
:10173000E02042F00102C3F8E020D3F8E03003F0EB
:1017400001030293029B142303934FF48813049321
:1017500003A90B4800F030FF22462146082000F084
:10176000FBFB082000F02EFC224621460A2000F058
:10177000F3FB0A2000F026FC08B010BD004402581C
:101780000000025872B6FEE700B59FB04C2200215F
:101790000BA804F083F92022002103A804F07EF9AD
:1017A000022001F02DF800230093384BDA6A22F072
:1017B0000102DA62DB6A03F001030093344B9A6999
:1017C00042F440429A619B6903F440430093009BBA
:1017D0002F4B9B6913F4005FFAD02E4BD3F8F42003
:1017E00042F00202C3F8F420D3F8F43003F002030D
:1017F0000193019B00230293254B9A6942F44042D6
:101800009A619B6903F440430293204BDA6A42F0E9
:101810000102DA62DB6A03F001030293029B1C4BB4
:101820009B6913F4005FFAD001230B934FF48033CC
:101830000C930223149315931693F0221792189386
:1018400019931A9308231B9300231C931D930BA831
:1018500001F000F8B0B93F2303930323049300235E
:101860000593082306934023079308934FF480625F
:1018700009920A93042103A801F052FC20B91FB079
:101880005DF804FBFFF77EFFFFF77CFF00040058C4
:10189000004802580044025808B5344B5B6913F401
:1018A000003F13D1BFF34F8FBFF36F8F2F4B002239
:1018B000C3F85022BFF34F8FBFF36F8F5A6942F4C2
:1018C00000325A61BFF34F8FBFF36F8F274B5B69B5
:1018D00013F4803F27D1254B0022C3F88420BFF3A7
:1018E0004F8FD3F88040C4F34E3000E01846C4F365
:1018F000C90243F6E07303EA401343EA82731B49CB
:10190000C1F860321346013A002BF2D1431E002881
:10191000ECD1BFF34F8F4B6943F480334B61BFF37E
:101920004F8FBFF36F8F00F0BFFAFFF72DFFFFF768
:10193000E9FE00F06BF900F0DDF90D4800F024F845
:101940003C210C4802F0CDFF0A4B1B68596A0A4B38
:1019500019600A4804F0F4F800F0E0FA084B186047
:101960001968084804F0ECF8EEE700BF00ED00E06D
:10197000380A0024EC090024E009002468BB0008B0
:10198000DC09002478BB000808B5054B1860054B3E
:101990001868002302221946806804F0E5F808BDA3
:1019A000E409002410000024022801D80120704717
:1019B00008B504F049F809230360002008BD0000C1
:1019C00010B5013801280AD814464FF0FF3392B2FF
:1019D0000748006803F01AFE40B9204610BD04F025
:1019E00033F8092303604FF0FF30F7E70520F5E7F0
:1019F000E4090024022801D80020704708B504F04B
:101A000023F8092303604FF0FF3008BD08B504F048
:101A10001BF8092303604FF0FF3008BD08B548B933
:101A20004FF0FF3301220848006803F057FE40B929
:101A3000012008BD04F008F8092303604FF0FF30CF
:101A4000F7E70520F5E700BFE409002408B5022800
:101A500004D84FF400534B60002008BD03F0F4FF9E
:101A600009230360F8E7000082B0074BD3F8F420A5
:101A700042F00202C3F8F420D3F8F43003F002037A
:101A80000193019B02B0704700440258FEE7FEE755
:101A9000FEE7FEE7FEE770477047704708B500F0C5
:101AA00031FA08BD08B5042000F09AFE08BD000018
:101AB00008B5102000F094FE024B1B6800225A6209
:101AC00008BD00BFEC09002408B5024802F055FD2E
:101AD00008BD00BFEC09002408B5024803F006F871
:101AE00008BD00BF380A00240120704708B503F084
:101AF000ABFF162303604FF0FF3008BD08B54FF071
:101B0000FF31FFF7F3FFFEE710B503460C4A0D491E
:101B10000D48006840B10C4800680344521A9342D3
:101B200006D8094A136010BD0748084C0460F2E764
:101B300003F08AFF0C2303604FF0FF30F3E700BF90
:101B40000000082400040000E8090024180B002409
:101B5000244B1B6803F00F03062B06D8214A136899
:101B600023F00F0343F0070313601F4B1A6842F082
:101B700001021A6000221A6119681C4A0A401A60A0
:101B8000184B1B6813F0080F06D0164A136823F091
:101B90000F0343F007031360134B00229A61DA61CD
:101BA0001A62134999621349D962134919635A6336
:101BB0009963DA6319645A64196821F48021196001
:101BC0001A660E4B1A680E4B1340B3F1005F03D236
:101BD0000C4B0122C3F808210B4B43F2D2021A60CE
:101BE000704700BF00200052004402587FEDF6EA23
:101BF000000202020000FF01800201010010005CEF
:101C00000000FFFF008000510040005200B58DB081
:101C10002422002103A803F041FF00230093019335
:101C2000029312484FF080420260032242608360B8
:101C30004FF0FF31C160036183610392012305937B
:101C4000099303A902F0E0FD50B900230093029329
:101C50006946064802F0AAFE28B90DB05DF804FBFB
:101C6000FFF790FDF1E7FFF78DFDF6E7EC090024A3
:101C700000B589B00023039304930593069307935B
:101C80000368B3F1804F02D009B05DF804FB164B36
:101C9000D3F8E82042F00102C3F8E820D3F8E820A6
:101CA00002F001020192019AD3F8E02042F0010211
:101CB000C3F8E020D3F8E03003F001030293029B65
:101CC00003230393022304930123079303A90748E3
:101CD00000F072FC002211461C2000F03DF91C208F
:101CE00000F070F9D0E700BF00440258000002582D
:101CF0007047000008B51748174B03604FF4E133F5
:101D0000436000238360C36003610C2242618361EE
:101D1000C36103624362836203F0D0FD70B90021A6
:101D20000C4803F047FE60B900210A4803F067FE43
:101D300050B9084803F01FFE48B908BDFFF722FD5F
:101D4000EDE7FFF71FFDEFE7FFF71CFDF1E7FFF7FA
:101D500019FDF2E7380A00240010014010B5B8B0B0
:101D60000446002133913491359136913791C02248
:101D700002A803F093FE22681F4B9A4201D038B0AC
:101D800010BD01220023CDE9022302A801F064FC6A
:101D900078BB1A4BD3F8F02042F01002C3F8F020C1
:101DA000D3F8F02002F010020092009AD3F8E0205D
:101DB00042F00102C3F8E020D3F8E03003F0010361
:101DC0000193019B4FF4C0633393022334930024A7
:101DD000359436940723379333A9094800F0ECFB78
:101DE00022462146252000F0B7F8252000F0EAF829
:101DF000C5E7FFF7C7FCCCE70010014000440258DC
:101E000000000258DFF834D0FFF7A2FE0C480D495D
:101E10000D4A002302E0D458C4500433C4188C4245
:101E2000F9D30A4A0A4C002301E013600432A242AB
:101E3000FBD303F00FFEFFF72FFD704700000824CF
:101E400000000024C0090024D4BF0008C0090024F9
:101E5000180B0024FEE70000104B1B780BB9012083
:101E6000704710B504464FF47A70B0FBF3F30C4A98
:101E70001068B0FBF3F000F0B3F868B90F2C01D98B
:101E800001200AE0002221464FF0FF3000F064F804
:101E9000044B1C60002000E0012010BD080000245D
:101EA000000000240C00002410B5032000F042F8CC
:101EB00001F02AF80F498B69C3F303230E4AD35C60
:101EC00003F01F03D8408B6903F00F03D35C03F0CA
:101ED0001F0320FA03F3094A1360094B18600F200F
:101EE000FFF7BAFF10B10124204610BD0446FFF7EA
:101EF000BBFDF9E7004402588CBB00080400002435
:101F000000000024034B1B78034A11680B44136044
:101F1000704700BF08000024CC0A0024014B186859
:101F2000704700BFCC0A0024014B1868000C7047B2
:101F30000010005C0649CB6823F4E0631B041B0C13
:101F4000000200F4E0600343024A1A43CA6070478B
:101F500000ED00E00000FA0500B5174BDB68C3F3A5
:101F60000223C3F1070CBCF1040F28BF4FF0040C8F
:101F700003F1040EBEF1060F14D9033B4FF0FF3EF0
:101F80000EFA0CFC21EA0C0199400EFA03F322EA46
:101F900003031943002807DB0901C9B2074B195491
:101FA0005DF804FB0023E9E700F00F000901C9B266
:101FB000034B1954F4E700BF00ED00E000E400E03B
:101FC00014ED00E0002807DB00F01F0240090123A8
:101FD0009340024A42F82030704700BF00E100E021
:101FE0000138B0F1807F0BD24FF0E0235861054AF1
:101FF000F02182F823100020986107221A617047AF
:102000000120704700ED00E070B50446FFF786FF41
:10201000002C00F09181054694F83530DBB2022B9C
:1020200006D080236365002384F83430012070BD1E
:1020300023688C498C4A934218BF8B4230D01832A7
:1020400093422DD0183293422AD01832934227D08F
:102050001832934224D01832934221D0183293423E
:102060001ED002F5567293421AD01832934217D0FE
:102070001832934214D01832934211D0183293423E
:102080000ED0183293420BD01832934208D0183237
:10209000934205D01A6822F00E021A60266809E001
:1020A0001A6822F01E021A602268536923F0800326
:1020B0005361266823686B496B4A934218BF8B4271
:1020C00042D0183293423FD0183293423CD018325B
:1020D000934239D01832934236D01832934233D0DB
:1020E0001832934230D002F5567293422CD01832F7
:1020F000934229D01832934226D01832934223D0EB
:102100001832934220D0183293421DD01832934295
:102110001AD01832934217D0544A934214D0143232
:10212000934211D0143293420ED0143293420BD00A
:102130001432934208D01432934205D014329342A1
:1021400002D01432934204D1226E136823F48073B8
:10215000136023684349444A934218BF8B422FD0EF
:10216000183293422CD01832934229D0183293421D
:1021700026D01832934223D01832934220D01832FE
:1021800093421DD002F55672934219D018329342F1
:1021900016D01832934213D01832934210D018320E
:1021A00093420DD0183293420AD01832934207D08E
:1021B0001832934204D01A6822F001021A6003E038
:1021C0001A6822F001021A60336813F0010F0ED072
:1021D000FFF7A4FE431B052BF6D9202363650323D9
:1021E00084F83530002384F8343001201FE7236859
:1021F0001C491D4A934218BF8B4239D01832934272
:1022000036D01832934233D01832934230D018323D
:1022100093422DD0183293422AD01832934227D0BD
:1022200002F55672934223D01832934220D01832CE
:1022300093421DD0183293421AD01832934217D0CD
:102240001832934214D01832934211D0183293426C
:102250000ED0A16DE36D03F01F02012393404B608C
:102260000DE000BF10000240280002400854025850
:10227000A16DE36D03F01F023F2393408B60236841
:102280002E492F4A934218BF8B4242D018329342B4
:102290003FD0183293423CD01832934239D0183292
:1022A000934236D01832934233D01832934230D012
:1022B00002F5567293422CD01832934229D018322C
:1022C000934226D01832934223D01832934220D022
:1022D000183293421DD0183293421AD018329342CA
:1022E00017D0184A934214D01432934211D01432AA
:1022F00093420ED0143293420BD01432934208D042
:102300001432934205D01432934202D014329342D5
:102310000BD1636EA26E5A60E36E33B11A6822F479
:1023200080721A60236F626F5A60012384F835301F
:10233000002084F834007AE6012078E6100002409C
:102340002800024008540258002800F0298108B5EE
:10235000024690F83530DBB2022B03D08023436570
:10236000012008BD0368904890498B4218BF834202
:102370000CBF0121002166D03030834263D0183079
:10238000834260D0183083425DD0183083425AD0E7
:102390001830834257D01830834254D000F556701D
:1023A000834250D0183083424DD0183083424AD0F7
:1023B0001830834247D01830834244D018308342CB
:1023C00041D0183083423ED0183083423BD0196848
:1023D00021F00E0119601368A0F5956073498B42D6
:1023E00018BF83426AD072498B4267D018318B4242
:1023F00064D018318B4261D018318B425ED01831D5
:102400008B425BD018318B4258D001F556718B420C
:1024100054D018318B4251D018318B424ED01831E4
:102420008B424BD018318B4248D018318B4245D06B
:1024300018318B4242D018318B423FD0196821F0BD
:10244000010119603EE0042082F8350081BB584A42
:1024500093422DD0183293422AD01832934227D07B
:102460001832934224D01832934221D0183293422A
:102470001ED002F5567293421AD01832934217D0EA
:102480001832934214D01832934211D0183293422A
:102490000ED0183293420BD01832934208D0183223
:1024A000934205D01A6822F001021A60002058E712
:1024B0001A6822F001021A60002052E7196821F020
:1024C000010119601368384838498B4218BF8342AC
:1024D00042D018318B423FD018318B423CD018315A
:1024E0008B4239D018318B4236D018318B4233D0E1
:1024F00018318B4230D001F556718B422CD01831F7
:102500008B4229D018318B4226D018318B4223D0F0
:1025100018318B4220D018318B421DD018318B429C
:102520001AD018318B4217D022498B4214D0143163
:102530008B4211D014318B420ED014318B420BD010
:1025400014318B4208D014318B4205D014318B42A8
:1025500002D014318B4217D1116E0B6823F48073B3
:102560000B60906DD36D03F01F0101238B4043601E
:10257000536E916E5960D36E33B1196821F4807136
:102580001960136F516F5960012382F835300023B1
:1025900082F83430136D2BB1104698470020E0E6E6
:1025A000012070470020DCE61000024028000240B5
:1025B000400002400854025870B582B000236EE01B
:1025C00085685E000324B44025EA0405CC68B44065
:1025D0002C438460446824EA0C0C4C68C4F3001457
:1025E0009C4044EA0C0444606CE0DD08083550F877
:1025F000256003F007044FEA840C0F2404FA0CF45E
:1026000026EA040E0C6904FA0CF444EA0E0440F8BD
:1026100025406FE0092400E0002404FA0EF42C4366
:102620000CF1020C6B4D45F82C404FF0B04425687E
:10263000D44325EA0206D1F804C01CF4801F01D05F
:1026400042EA05064FF0B0452E606D6804EA0506C3
:10265000D1F804C01CF4001F01D042EA05064FF077
:10266000B0456E60D5F8845004EA0506D1F804C080
:102670001CF4003F01D042EA05064FF0B045C5F812
:102680008460D5F880502C404E6816F4803F01D00D
:1026900042EA05044FF0B042C2F8804001330A68B4
:1026A00032FA03F400F093804FF0010C0CFA03FCB3
:1026B0001CEA0202F2D04C6804F00304013C012C35
:1026C0007FF67EAF4C6804F00304032C0CD0C46882
:1026D0005D004FF0030C0CFA05FC24EA0C0C8C682E
:1026E000AC4044EA0C04C4604C6804F00304022CBF
:1026F0003FF47BAF04684FEA430E4FF0030C0CFA33
:102700000EFC24EA0C0C4C6804F0030404FA0EF4EA
:1027100044EA0C0404604C6814F4403FBED02E4CD4
:10272000D4F8F45045F00205C4F8F450D4F8F4405D
:1027300004F002040194019C4FEA930C0CF1020591
:10274000244C54F8255003F003044FEA840E0F2460
:1027500004FA0EF425EA0405204CA0423FF45CAFD5
:1027600004F58064A04222D004F58064A04220D009
:1027700004F58064A0421ED004F58064A0421CD001
:1027800004F58064A0421AD004F58064A04218D0F9
:1027900004F58064A04216D004F58064A04214D0F1
:1027A00004F58064A0423FF435AF0A2435E70124E4
:1027B00033E7022431E703242FE704242DE705241F
:1027C0002BE7062429E7072427E7082425E702B09A
:1027D00070BD00BF000400580044025800000258B9
:1027E00008B54FF0B043D3F88830034200D108BD9C
:1027F0004FF0B043C3F88800FFF77AFAF7E700001C
:10280000134BDB6813F0040F07D1114BDB6803F0A7
:10281000070383421AD00120704710B50C4AD368D1
:1028200023F007031843D060FFF778FB0446084BFA
:102830005B6813F4005F07D1FFF770FB001BB0F576
:102840007A7FF4D9012000E0002010BD00207047FD
:1028500000480258002800F0398338B50446036860
:1028600013F0010F25D0944A136903F03803926ADC
:10287000102B15D0182B0FD06368B3F5803F3FD0D5
:10288000002B53D18C4B1A6822F480321A601A68DC
:1028900022F480221A6038E002F00302022AEBD10F
:1028A000854B1B6813F4003F03D06368002B00F0D6
:1028B0000F83236813F0020F00F0A1807E4A136992
:1028C000926A13F038035AD0182B55D0E368002BC6
:1028D00000F0DE8078490A6822F0190213430B6089
:1028E000FFF71CFB0546744B1B6813F0040F40F008
:1028F000AD80FFF713FB401B0228F4D90320EEE262
:102900006D4A136843F48033136063682BB3FFF799
:1029100005FB0546684B1B6813F4003FC9D1FFF760
:10292000FDFA401B6428F5D90320D8E2B3F5A02FA7
:1029300009D0614B1A6822F480321A601A6822F4B6
:1029400080221A60E1E75C4B1A6842F480221A6028
:102950001A6842F480321A60D7E7FFF7DFFA0546BB
:10296000554B1B6813F4003FA3D0FFF7D7FA401B69
:102970006428F5D90320B2E212F0030FA6D14E4B22
:102980001B6813F0040F03D0E368002B00F0A28251
:10299000494A136823F01903E1680B431360FFF7FA
:1029A000BDFA0546444B1B6813F0040F06D1FFF730
:1029B000B5FA401B0228F5D9032090E2FFF7B4FADC
:1029C00041F20303984212D82269402A07D03A49BB
:1029D0004B6823F47C3343EA02334B600FE0364A02
:1029E000536823F47C3343F40033536007E0324AE6
:1029F000536823F0FE43216943EA0163536023686F
:102A000013F0100F00F088802B4A136903F038038D
:102A1000926A082B56D0182B50D0E369002B00F097
:102A2000B880254A136843F080031360FFF776FAF5
:102A30000546214B1B6813F4807F40F08880FFF728
:102A40006DFA401B0228F4D9032048E2FFF76CFA24
:102A500041F20303984212D82269402A07D016494E
:102A60004B6823F47C3343EA02334B60C7E7124AD6
:102A7000536823F47C3343F400335360BFE70E4ABA
:102A8000536823F0FE43216943EA01635360B6E7CC
:102A9000094A136823F001031360FFF73FFA054664
:102AA000054B1B6813F0040FA9D0FFF737FA401B42
:102AB0000228F5D9032012E20044025802F0030272
:102AC000012AAAD1A14B1B6813F4807F03D0E369CC
:102AD000802B40F00182FFF727FA41F2030398426E
:102AE00012D8226A202A07D098494B6823F0F8436D
:102AF00043EA82634B600FE0944A536823F0F84343
:102B000043F08043536007E0904AD36823F07C533E
:102B1000216A43EA0163D360236813F0080F60D091
:102B20006369002B49D0894A536F43F0010353670F
:102B3000FFF7F4F90546854B5B6F13F0020F50D198
:102B4000FFF7ECF9401B0228F5D90320C7E1FFF796
:102B5000EBF941F20303984212D8226A202A07D0E7
:102B60007A494B6823F0F84343EA82634B60D3E72A
:102B7000764A536823F0F84343F080435360CBE731
:102B8000724AD36823F07C53216A43EA0163D3601D
:102B9000C2E76E4A136823F080031360FFF7BEF9A3
:102BA00005466A4B1B6813F4807FB5D0FFF7B6F972
:102BB000401B0228F5D9032091E1644A536F23F0AA
:102BC00001035367FFF7AAF90546604B5B6F13F0EB
:102BD000020F06D0FFF7A2F9401B0228F5D9032007
:102BE0007DE1236813F0200F29D0A3699BB1574AD8
:102BF000136843F480531360FFF790F90546534B75
:102C00001B6813F4005F1AD1FFF788F9401B0228F4
:102C1000F5D9032063E14D4A136823F48053136010
:102C2000FFF77CF90546494B1B6813F4005F06D09B
:102C3000FFF774F9401B0228F5D903204FE1236800
:102C400013F0040F21D1636A002B00F047813F4A43
:102C5000126902F03802182A00F0EE80022B79D0B7
:102C60003A4A136823F080731360FFF757F904465C
:102C7000364B1B6813F0007F00F0DC80FFF74EF945
:102C8000001B0228F4D9032029E1314A136843F4D8
:102C900080731360FFF742F905462D4B1B6813F450
:102CA000807F06D1FFF73AF9401B6428F5D903204D
:102CB00015E1A368012B0AD00BBB244B1A6F22F03D
:102CC00001021A671A6F22F004021A6704E01F4A11
:102CD000136F43F001031367A36833B3FFF71EF9C3
:102CE00005461A4B1B6F13F0020FACD1FFF716F914
:102CF000401B41F288339842F3D90320EFE0052BC3
:102D000009D0124B1A6F22F001021A671A6F22F0D3
:102D100004021A67E0E70D4B1A6F42F004021A67CB
:102D20001A6F42F001021A67D6E7FFF7F7F8054677
:102D3000064B1B6F13F0020F85D0FFF7EFF8401B17
:102D400041F288339842F3D90320C8E00044025886
:102D500000480258694A136823F080731360FFF734
:102D6000DDF80546654B1B6813F0007F06D0FFF7C2
:102D7000D5F8401B0228F5D90320B0E05F4B996AD3
:102D80005F4A0A40A16AE06A41EA00110A439A6276
:102D9000226B013AC2F30802616B0139490289B220
:102DA0000A43A16B0139090401F4FE010A43E16BF6
:102DB0000139090601F0FE410A431A63DA6A22F07A
:102DC0000102DA62596B4F4A0A40A16C42EAC10221
:102DD0005A63DA6A22F00C02216C0A43DA62DA6A78
:102DE00022F00202616C0A43DA62DA6A42F480324B
:102DF000DA62DA6A42F40032DA62DA6A42F4802293
:102E0000DA62DA6A42F00102DA621A6842F080722B
:102E10001A60FFF783F80446384B1B6813F0007FF5
:102E200006D1FFF77BF8001B0228F5D9032056E0F6
:102E3000002054E0002052E0304A916A106B012BD0
:102E40004ED001F00303A26A93424BD1C1F30511A6
:102E5000E36A994248D1C0F30802236B013B9A42CE
:102E600044D1C0F34622636B013B9A4240D1C0F388
:102E70000642A36B013B9A423CD1C0F30660E36B70
:102E8000013B984238D11D4B5B6BC3F3CC03A26C62
:102E90009A4201D1002022E0184AD36A23F00103AC
:102EA000D362FFF73BF80546FFF738F8A842FBD09E
:102EB000124A516B134B0B40A16C43EAC10353639D
:102EC000D36A43F00103D362002008E00120704779
:102ED000012004E0012002E0012000E0002038BDD4
:102EE0000120FCE70120FAE70120F8E70120F6E7DE
:102EF0000120F4E70120F2E70120F0E70044025846
:102F00000CFCFFFF0700FFFFF8B57E4B1B6903F0C9
:102F10003803102B00F0F280182B10D013B17A4C2C
:102F20002046F8BD774B1B6813F0200F00F0E880B7
:102F3000744B1868C0F3C100744CC440F0E7714B87
:102F40009D6A05F003059C6AC4F30514D86A00F075
:102F500001005B6BC3F3CC0303FB00F0FDF786FAC3
:102F60000646002CDCD0012D76D0022D00F0A48086
:102F70000DB32046FDF77AFA01466548FDF782FB5E
:102F80000446604B186BC0F30800FDF76FFA054666
:102F90004FF064513046FDF7C1FA01462846FDF76F
:102FA000B5F94FF07E51FDF7B1F901462046FDF726
:102FB000B5FA044671E0534B1B6813F0200F29D07B
:102FC000504F3B68C3F3C1035048D840FDF74EFA59
:102FD00005462046FDF74AFA01462846FDF752FB12
:102FE0000446386BC0F30800FDF740FA05464FF081
:102FF00064513046FDF792FA01462846FDF786F9FE
:103000004FF07E51FDF782F901462046FDF786FA22
:10301000044642E02046FDF729FA01463D48FDF707
:1030200031FB0446374B186BC0F30800FDF71EFA5E
:1030300005464FF064513046FDF770FA01462846C8
:10304000FDF764F94FF07E51FDF760F90146204627
:10305000FDF764FA044620E02046FDF707FA014632
:103060002B48FDF70FFB0446264B186BC0F30800F6
:10307000FDF7FCF905464FF064513046FDF74EFA76
:1030800001462846FDF742F94FF07E51FDF73EF923
:1030900001462046FDF742FA04461A4B1B6BC3F368
:1030A0004623581CFDF7E2F901462046FDF7EAFAEF
:1030B000FDF784FB044633E72046FDF7D7F90146C8
:1030C0001548FDF7DFFA04460E4B186BC0F30800F5
:1030D000FDF7CCF905464FF064513046FDF71EFA76
:1030E00001462846FDF712F94FF07E51FDF70EF923
:1030F00001462046FDF712FA0446CEE7074C0FE7DB
:10310000024C0DE70044025800093D000090D00336
:103110000024744A0024744C0024F44A00127A00FB
:10312000002800F0328170B50D4604469B4B1B68A9
:1031300003F00F038B420BD2984A136823F00F035E
:103140000B431360136803F00F038B4240F01F81A1
:10315000236813F0040F0CD02269914B9B6903F094
:1031600070039A4205D98E498B6923F070031A4384
:103170008A61236813F0080F0CD06269884BDB6901
:1031800003F070039A4205D98549CB6923F0700397
:103190001A43CA61236813F0100F0CD0A269804B48
:1031A000DB6903F4E0639A4205D97D49CB6923F4D6
:1031B000E0631A43CA61236813F0200F0CD0E26960
:1031C000774B1B6A03F070039A4205D974490B6A66
:1031D00023F070031A430A62236813F0020F0CD025
:1031E000E2686F4B9B6903F00F039A4205D96C4963
:1031F0008B6923F00F031A438A61236813F0010FD0
:1032000041D0674A936923F47063A1680B439361CB
:103210006368022B0AD0032B27D0012B2CD0604AE5
:10322000126812F0040F06D10120ADE0126812F40A
:10323000003F00F0AE805A490A6922F007021343AA
:103240000B61FEF76BFE0646554B1B6903F0380316
:103250006268B3EBC20F16D0FEF760FE801B41F22E
:1032600088339842F0D903208EE04D4A126812F05C
:10327000007FE0D1012087E0494A126812F4807F84
:10328000D9D1012080E0236813F0020F0CD0E2684E
:10329000434B9B6903F00F039A4205D240498B6967
:1032A00023F00F031A438A613C4B1B6803F00F03A2
:1032B000AB420AD9394A136823F00F032B4313603A
:1032C000136803F00F03AB4265D1236813F0040FBA
:1032D0000CD02269324B9B6903F070039A4205D2ED
:1032E0002F498B6923F070031A438A61236813F016
:1032F000080F0CD062692A4BDB6903F070039A4215
:1033000005D22749CB6923F070031A43CA612368A9
:1033100013F0100F0CD0A269214BDB6903F4E063BA
:103320009A4205D21E49CB6923F4E0631A43CA616D
:10333000236813F0200F0CD0E269194B1B6A03F0CD
:1033400070039A4205D216490B6A23F070031A43A0
:103350000A62FFF7D9FD12498B69C3F30323114AAF
:10336000D35C03F01F03D8408B6903F00F03D35CD9
:1033700003F01F0320FA03F30B4A13600B4B186092
:103380000B4B1868FEF768FD70BD012070470120E7
:10339000FAE70120F8E70120F6E700BF002000521D
:1033A000004402588CBB00080400002400000024E4
:1033B0000C00002408B5FFF7A7FD0B4A9369C3F37F
:1033C00003230A49CB5C03F01F0320FA03F392693D
:1033D00002F00F02885C00F01F0023FA00F0044A9C
:1033E0001060044A136008BD004402588CBB0008FA
:1033F000040000240000002408B5FFF7DBFF054BA4
:10340000DB69C3F30213044AD35C03F01F03D84003
:1034100008BD00BF004402588CBB000808B5FFF788
:10342000C9FF054BDB69C3F30223044AD35C03F0F5
:103430001F03D84008BD00BF004402588CBB0008E1
:10344000404B9B6A03F00303032B79D070B505460C
:103450000E463C4A136823F080631360FEF75EFD5E
:103460000446384B1B6813F0006F06D0FEF756FD7C
:10347000031B022BF5D9032070BD324B9A6A22F44C
:103480007C32296842EA01329A626A68013AC2F3E0
:103490000802A9680139490289B20A43E968013979
:1034A000090401F4FE010A4329690139090601F002
:1034B000FE410A439A63DA6A22F0C00269690A434C
:1034C000DA62DA6A22F02002A9690A43DA62DA6A69
:1034D00022F01002DA62D96B1B4A0A40E96942EA1B
:1034E000C102DA63DA6A42F01002DA62C6B91A4639
:1034F000DB6A43F40023D362124A136843F080630B
:103500001360FEF70BFD04460E4B1B6813F0006FB3
:1035100014D1FEF703FD001B0228F5D90320ABE709
:10352000012E05D0074AD36A43F40013D362E3E7C0
:10353000044AD36A43F48013D362DDE700209BE79B
:1035400001207047004402580700FFFF404B9B6A70
:1035500003F00303032B79D070B505460E463C4AB1
:10356000136823F080531360FEF7D8FC0446384BF1
:103570001B6813F0005F06D0FEF7D0FC031B022B84
:10358000F5D9032070BD324B9A6A22F07C7229680B
:1035900042EA01529A626A68013AC2F30802A968D3
:1035A0000139490289B20A43E9680139090401F481
:1035B000FE010A4329690139090601F0FE410A4367
:1035C0001A64DA6A22F4406269690A43DA62DA6AE2
:1035D00022F40072A9690A43DA62DA6A22F480727C
:1035E000DA62596C1B4A0A40E96942EAC1025A642C
:1035F000DA6A42F48072DA62C6B91A46DB6A43F4C8
:103600008003D362124A136843F080531360FEF7BD
:1036100085FC04460E4B1B6813F0005F14D1FEF7C7
:103620007DFC001B0228F5D90320ABE7012E05D055
:10363000074AD36A43F08073D362E3E7044AD36A4C
:1036400043F40003D362DDE700209BE701207047CD
:10365000004402580700FFFFF8B50446036813F062
:10366000006F30D0836EB3F5001F26D00ED8EBB1BB
:10367000B3F5801F07D102210830FFF7E1FE0546B0
:1036800045B12E4621E0012635461EE0B3F5401F28
:1036900009D10025984A136D23F44013A16E0B4302
:1036A0001365002611E0012635460EE0924AD36AE2
:1036B00043F40033D3620025ECE702212830FFF702
:1036C00045FF0546DCE700263546236813F4807F76
:1036D00014D0A36D042B32D8DFE803F003232A08AB
:1036E0000800854AD36A43F40033D36255BB824A4B
:1036F000136D23F00703A16D0B431365236813F4C7
:10370000007F31D0E36D802B4CD020D8002B43D0EC
:10371000402B19D1002104F10800FFF791FE054666
:103720001AE0002104F10800FFF78AFE0546DDE7F4
:10373000002104F12800FFF709FF0546D6E701261E
:103740003546DBE72E46D9E7012635460CE0C02B8F
:1037500002D0B3F5807F1CD15DBB674A136D23F4A3
:10376000E073E16D0B431365236813F4806F46D05B
:10377000D4F8A830B3F5800F39D01FD88BB3B3F588
:10378000001F18D1002104F10800FFF759FE05467B
:103790001AE001263546E7E7574AD36A43F4003377
:1037A000D362D9E7002104F12800FFF7CFFE0546D8
:1037B000D2E72E46D8E70126354620E0B3F5C00F04
:1037C00002D0B3F5000F09D1C5B94B4A936D23F46C
:1037D0006003D4F8A8100B43936510E0012635462A
:1037E0000DE0454AD36A43F40033D362ECE700218D
:1037F00004F12800FFF7AAFE0546E5E72E462368F8
:1038000013F4006F24D0D4F8AC30B3F1007F42D071
:103810000ED8002B39D0B3F1807F06D1002104F1FE
:103820000800FFF70DFE054608E0012635460FE0CB
:10383000B3F1407F02D0B3F1806F23D1002D31D19D
:103840002D4A936D23F0E063D4F8AC100B439365DD
:10385000236813F0007F2ED0E36C202B40D026D8B5
:1038600033B1102B20D1244AD36A43F40033D362FE
:10387000002D3CD1204AD36C23F03003E16C0B4384
:10388000D36418E001263546E2E71B4AD36A43F4C5
:103890000033D362D2E7002104F12800FFF756FE7F
:1038A0000546CBE72E46D3E70126354603E0302B0D
:1038B000DED001263546236813F4805F2DD0236EB9
:1038C000B3F5005F4FD019D8002B46D0B3F5805F19
:1038D0000FD1002104F10800FFF7B2FD054613E007
:1038E000022104F10800FFF7ABFD0546C0E72E46B4
:1038F000E1E70126354610E000440258B3F5405F89
:1039000002D0B3F5804F25D1002D33D1774A136D06
:1039100023F4E043216E0B431365236813F4005F27
:1039200038D0636EB3F5003F53D028D843B1B3F518
:10393000803F21D1012104F10800FFF781FD0546F8
:10394000002D4DD1694A136D23F4E023616E0B43C2
:1039500013651FE001263546DFE7644AD36A43F466
:103960000033D362D0E7002104F12800FFF7EEFD19
:103970000546C9E72E46D0E7012635460AE0B3F5ED
:10398000802FDDD0B3F5A02FDAD0B3F5403FD7D0EC
:1039900001263546236813F4804F31D0D4F8B03077
:1039A000B3F1005F45D020D843B1B3F1805F19D1A6
:1039B000012104F10800FFF743FD0546002D3FD12A
:1039C0004A4A936D23F0E043D4F8B0100B4393655B
:1039D00016E0012104F12800FFF7B8FD0546AFE726
:1039E0002E46D7E7012635460AE0B3F1804FE5D0F1
:1039F000B3F1A04FE2D0B3F1405FDFD001263546EE
:103A0000236813F4004F09D0236FB3F1805F19D0FE
:103A1000B3F1005F24D0D3B101263546236813F0FB
:103A2000807F33D0A36C032B5BD8DFE803F0272221
:103A30005327012104F12800FFF788FD0546BDE763
:103A40002E46DDE7294AD36A43F40033D36275B9C1
:103A5000264A136D23F04053216F0B431365DDE7B6
:103A6000012104F10800FFF7EBFC0546EFE72E46C5
:103A7000D4E71E4AD36A43F40033D362A5BB1B4A82
:103A8000D36C23F00303A16C0B43D364236813F4BA
:103A9000800F2DD1236813F0010F00F0A580E36F94
:103AA000282B00F29F80DFE803F08D9D9D9D9D9D5A
:103AB0009D9D879D9D9D9D9D9D9D969D9D9D9D9D53
:103AC0009D9D8D9D9D9D9D9D9D9D8D9D9D9D9D9D46
:103AD0009D9D8D00022104F10800FFF7B1FC054611
:103AE000CCE701263546D1E72E46CFE70044025801
:103AF000914A136843F480731360FEF70FFA074688
:103B00008D4B1B6813F4807F05D1FEF707FAC01BAD
:103B10006428F5D90325002D4AD1884B1B6FD4F8B2
:103B2000B420534013F4407F0CD0844B1A6F22F41E
:103B30004072196F41F480311967196F21F4803197
:103B400019671A67D4F8B430B3F5807F15D08DBBF0
:103B5000D4F8B43003F44072B2F5407F1ED0774AF7
:103B6000136923F47C53136174490B6FD4F8B420A8
:103B7000C2F30B0213430B678CE7FEF7CFF907463E
:103B80006E4B1B6F13F0020FE1D1FEF7C7F9C01B9C
:103B900041F288339842F3D90325D8E76748026990
:103BA00022F47C52664901EA131313430361DBE7F5
:103BB0002E466FE72E466DE7012104F10800FFF75E
:103BC0003FFC0546E5B95D4A536D23F03803E16FCC
:103BD0000B43536508E0012104F12800FFF7B6FC10
:103BE0000546EFE701263546236813F0020F17D08C
:103BF000A36F052B28D8DFE803F00B05200B0B0B78
:103C00002E46F1E7012104F10800FFF719FC0546F3
:103C1000EDB94A4A536D23F00703A16F0B43536577
:103C2000236813F0040F23D0D4F89430052B45D823
:103C3000DFE803F0150F3D151515012104F12800EB
:103C4000FFF784FC0546E3E701263546E8E72E4604
:103C5000E6E7012104F10800FFF7F2FB054685BB0A
:103C6000364A936D23F00703D4F894100B43936501
:103C7000236813F0200F34D0D4F89030B3F1005FF4
:103C80004ED023D843B1B3F1805F1CD1002104F1A1
:103C90000800FFF7D5FB0546002D48D1274A536D94
:103CA00023F0E043D4F890100B43536519E0012151
:103CB00004F12800FFF74AFC0546D0E70126354607
:103CC000D6E72E46D4E7012635460AE0B3F1804F09
:103CD000E2D0B3F1A04FDFD0B3F1405FDCD00126DA
:103CE0003546236813F0400F37D0D4F89C30B3F535
:103CF000006F53D026D843B1B3F5806F19D100219E
:103D000004F10800FFF79CFB0546002D4DD10B4A3E
:103D1000936D23F4E053D4F89C100B4393651CE09F
:103D2000022104F12800FFF711FC0546B4E72E46F6
:103D3000D7E70126354610E00048025800440258F3
:103D4000CFFFFF00B3F5805FDFD0B3F5A05FDCD01D
:103D5000B3F5406FD9D001263546236813F0800FA4
:103D600033D0D4F8A030B3F5804F00F0A38021D831
:103D700043B1B3F5005F1AD1002104F10800FFF749
:103D80005FFB0546002D40F09C80814A936D23F433
:103D90006043D4F8A0100B43936516E0022104F1B0
:103DA0002800FFF7D3FB0546AFE72E46D5E70126EF
:103DB00035460AE0B3F5004FE4D0B3F5204FE1D02B
:103DC000B3F5C04FDED001263546236813F0080F47
:103DD0000CD0D4F88430B3F5805F74D06C4A536D46
:103DE00023F44053D4F884100B435365236813F035
:103DF000100F0CD0D4F89830B3F5807F6CD0644AA3
:103E0000936D23F44073D4F898100B4393652368A3
:103E100013F4002F0BD0D4F8A430B3F5803F74D046
:103E2000B3F5003F67D0002B5FD0012635462368ED
:103E300013F4802F0CD0D4F88830B3F5001F7CD059
:103E4000B3F5401F6FD0B3F5801F67D0012635460C
:103E5000236813F4803F08D0236D002B76D0B3F590
:103E6000803F00F0818001263546236813F0005F13
:103E700040F08380236813F4003F00F08E80D4F874
:103E80008030B3F5807F00F0EC8040F28380B3F5A2
:103E9000007F03D0B3F5407F40F0E180002D40F07B
:103EA000E6803B4A536D23F44073D4F880100B43F3
:103EB000536572E0022104F12800FFF747FB054635
:103EC00060E72E4681E7022104F12800FFF73EFB60
:103ED000002883D0012681E7022104F12800FFF7A2
:103EE00035FB00288BD0012689E7002104F108006A
:103EF000FFF7A6FA05467DB9254A936D23F44033B2
:103F0000D4F8A4100B43936591E7022104F1280033
:103F1000FFF71CFB0546EEE72E4688E71C4AD36AEE
:103F200043F40033D3627DB9194A536D23F440132F
:103F3000D4F888100B4353658AE7012104F1280067
:103F4000FFF704FB0546EEE72E4681E7104AD36AE9
:103F500043F40033D36275B90D4AD36C23F4803334
:103F6000216D0B43D36480E7022104F10800FFF7C1
:103F700067FA0546EFE72E4677E7022104F12800AD
:103F8000FFF7E4FA00283FF475AF012672E700BF9F
:103F900000440258002B81D00126236813F4801FAF
:103FA00006D04F4A136D23F00043616F0B43136536
:103FB000236813F0805F07D0494A136923F48043D4
:103FC000D4F8B8100B431361236813F4001F06D014
:103FD000434A136D23F08073E16E0B43136523682E
:103FE00013F0804F09D03E4B1A6922F400421A6147
:103FF0001A69D4F8BC100A431A612368002B06DA48
:10400000374AD36C23F04053616D0B43D36423686C
:1040100013F4000F07D0324A536D23F44003D4F851
:104020008C100B435365636813F0010F21D1636853
:1040300013F0020F26D1636813F0040F2BD16368CD
:1040400013F0080F30D1636813F0100F35D1636897
:1040500013F0200F3AD106B101263046F8BD0126F3
:104060009BE71F4AD36A43F40033D36216E72E4618
:1040700093E7002104F10800FFF7E2F90028D6D009
:104080000646D4E7012104F10800FFF7D9F900281A
:10409000D1D00646CFE7022104F10800FFF7D0F99E
:1040A0000028CCD00646CAE7002104F12800FFF71B
:1040B0004DFA0028C7D00646C5E7012104F12800C3
:1040C000FFF744FA0028C2D00646C0E7022104F1F7
:1040D0002800FFF73BFA0028BDD00646BBE700BF2B
:1040E0000044025808B5FFF765F9054B1B6AC3F396
:1040F0000213044AD35C03F01F03D84008BD00BF7D
:10410000004402588CBB00082DE9F0410446864B60
:104110009D6A9E6AC6F30536D86AC0F30010DB6B51
:10412000C3F3CC0303FB00F0FCF7A0F9002E00F072
:10413000F58005F003050746012D79D0022D00F02A
:10414000CB800DB33046FCF791F901467748FCF778
:1041500099FA0546744B986BC0F30800FCF786F992
:1041600006464FF064513846FCF7D8F90146304610
:10417000FCF7CCF84FF07E51FCF7C8F80146284612
:10418000FCF7CCF9054674E0674B1B6813F0200F71
:104190002CD0DFF89481D8F80030C3F3C103644811
:1041A000D840FCF763F905463046FCF75FF9014655
:1041B0002846FCF767FA0546D8F83800C0F308002F
:1041C000FCF754F906464FF064513846FCF7A6F95F
:1041D00001463046FCF79AF84FF07E51FCF796F80E
:1041E00001462846FCF79AF9054642E03046FCF7BE
:1041F0003DF901464F48FCF745FA05464A4B986B96
:10420000C0F30800FCF732F906464FF06451384617
:10421000FCF784F901463046FCF778F84FF07E5100
:10422000FCF774F801462846FCF778F9054620E0CB
:104230003046FCF71BF901463C48FCF723FA0546DB
:10424000394B986BC0F30800FCF710F906464FF0A5
:1042500064513846FCF762F901463046FCF756F8DF
:104260004FF07E51FCF752F801462846FCF756F90C
:1042700005462D4EB06BC0F34620FCF7F7F84FF023
:104280007E51FCF743F801462846FCF7FBF9FCF7A2
:1042900095FA2060B06BC0F30640FCF7E7F84FF0EA
:1042A0007E51FCF733F801462846FCF7EBF9FCF7A2
:1042B00085FA6060B06BC0F30660FCF7D7F84FF08A
:1042C0007E51FCF723F801462846FCF7DBF9FCF7A2
:1042D00075FAA060BDE8F0813046FCF7C7F80146EA
:1042E0001548FCF7CFF905460F4B986BC0F3080053
:1042F000FCF7BCF806464FF064513846FCF70EF95F
:1043000001463046FCF702F84FF07E51FBF7FEFF06
:1043100001462846FCF702F90546AAE70023236078
:104320006360A360D6E700BF004402580024744ACB
:104330000090D0030024744C0024F44A2DE9F0418D
:104340000446864B9D6A9E6AC6F30556D86AC0F33A
:1043500000205B6CC3F3CC0303FB00F0FCF786F892
:10436000002E00F0F58005F003050746012D79D0F9
:10437000022D00F0CB800DB33046FCF777F80146F4
:104380007748FCF77FF90546744B186CC0F30800BA
:10439000FCF76CF806464FF064513846FCF7BEF85F
:1043A00001463046FBF7B2FF4FF07E51FBF7AEFF00
:1043B00001462846FCF7B2F8054674E0674B1B68D7
:1043C00013F0200F2CD0DFF89481D8F80030C3F31D
:1043D000C1036448D840FCF749F805463046FCF76D
:1043E00045F801462846FCF74DF90546D8F8400047
:1043F000C0F30800FCF73AF806464FF0645138461F
:10440000FCF78CF801463046FBF780FF4FF07E51F9
:10441000FBF77CFF01462846FCF780F8054642E0A2
:104420003046FCF723F801464F48FCF72BF90546C8
:104430004A4B186CC0F30800FCF718F806464FF01A
:1044400064513846FCF76AF801463046FBF75EFFD8
:104450004FF07E51FBF75AFF01462846FCF75EF805
:10446000054620E03046FCF701F801463C48FCF7E1
:1044700009F90546394B186CC0F30800FBF7F6FF45
:1044800006464FF064513846FCF748F8014630467E
:10449000FBF73CFF4FF07E51FBF738FF0146284603
:1044A000FCF73CF805462D4E306CC0F34620FBF778
:1044B000DDFF4FF07E51FBF729FF01462846FCF750
:1044C000E1F8FCF77BF92060306CC0F30640FBF7A5
:1044D000CDFF4FF07E51FBF719FF01462846FCF750
:1044E000D1F8FCF76BF96060306CC0F30660FBF745
:1044F000BDFF4FF07E51FBF709FF01462846FCF750
:10450000C1F8FCF75BF9A060BDE8F0813046FBF72D
:10451000ADFF01461548FCF7B5F805460F4B186C82
:10452000C0F30800FBF7A2FF06464FF0645138467F
:10453000FBF7F4FF01463046FBF7E8FE4FF07E51F3
:10454000FBF7E4FE01462846FBF7E8FF0546AAE72D
:10455000002323606360A360D6E700BF00440258D5
:104560000024744A0090D0030024744C0024F44AC0
:104570007047704770477047704770B504460368CE
:10458000DE681D6915F0020F10D016F0020F0DD075
:104590006FF002021A610123037703689B6913F02D
:1045A000030F64D0FFF7E6FF0023237715F0040F15
:1045B00012D016F0040F0FD023686FF004021A61B6
:1045C0000223237723689B6913F4407F55D020464C
:1045D000FFF7D0FF0023237715F0080F12D016F055
:1045E000080F0FD023686FF008021A6104232377A5
:1045F0002368DB6913F0030F46D02046FFF7BAFFAC
:104600000023237715F0100F12D016F0100F0FD0E3
:1046100023686FF010021A61082323772368DB698F
:1046200013F4407F37D02046FFF7A4FF0023237701
:1046300015F0010F02D016F0010F33D115F4025F0F
:1046400002D016F0800F35D115F4807F02D016F01D
:10465000800F37D115F0400F02D016F0400F39D13E
:1046600015F0200F02D016F0200F3BD170BDFFF7E0
:1046700080FF2046FFF77FFF96E72046FFF779FF90
:104680002046FFF778FFA5E72046FFF772FF204698
:10469000FFF771FFB4E72046FFF76BFF2046FFF7F7
:1046A0006AFFC3E723686FF001021A612046FFF733
:1046B0005FFFC3E723686FF402521A61204600F0DF
:1046C000C6F9C1E723686FF480721A61204600F0D2
:1046D000BFF9BFE723686FF040021A612046FFF779
:1046E0004BFFBDE723686FF020021A61204600F0FF
:1046F000ADF9BBE730B503683D4A904214BF4FF0B7
:10470000000E4FF0010EB0F1804F14BF72464EF014
:104710000102AAB9374CA04214BF00240124364D2F
:10472000A8420DD064B904F1804404F58234A0425B
:1047300014BF0024012405F50065A84200D01CB177
:1047400023F070034C68234312BB2A4A904214BFE3
:1047500000220122284CA0421AD0CAB902F180429C
:1047600002F58232904214BF0022012204F5006457
:10477000A0420DD062B9214A904214BF002201220A
:1047800004F59A34A04203D012B91D4A904204D1D4
:1047900023F4407CCB6843EA0C0323F080034A698E
:1047A000134303608A68C2620A688262154A9042B3
:1047B00014BF73464EF0010363B9104B984214BF07
:1047C0000023012302F57052904203D013B90C4B21
:1047D000984201D10B69036301234361036913F01C
:1047E000010F03D0036923F00103036130BD00BF53
:1047F0000000014000080040000400400044014067
:104800000048014000040140002852D070B50D4618
:10481000044690F83D30002B46D0022384F83D300A
:1048200022689168244B0B409360214651F8040B99
:10483000FFF760FF206881688369026A2E680E4373
:104840001E491940AB68D5F818C043EA0C2343EA67
:10485000010C1B4B0CEA0303E968D5F81CC041EAC4
:104860000C2119432B6A1B03D5F810C043EA0C1323
:104870000B4322F0AA016A686D6942EA05120A43F5
:10488000866021688B6123681A62012384F84830AE
:1048900084F83E3084F83F3084F8443084F8453062
:1048A00084F83D30002070BD80F83C30FDF7E0F921
:1048B000B3E70120704700BFF8BFFEFFFCFCFFFF1D
:1048C0000303FFFF01F01F01012303FA01FC036A48
:1048D00023EA0C030362036A02FA01F10B43036249
:1048E000704738B5044690F83E30DBB290F83F2070
:1048F0005FFA82FC90F84420D0B294F845200D462F
:10490000B1B9012808BF012B47D1022384F83E30FA
:1049100084F844307DB3042D39D001220021206871
:10492000FFF7D0FF012204212068FFF7CBFF27E02B
:10493000D2B2042914D0BCF1010F08BF012B30D131
:10494000013A18BF012201282DD162BB022384F84D
:104950003E3084F83F3084F8443084F84530D9E75D
:10496000012A08BFBCF1010F19D1022384F83F309E
:1049700084F84530CEE7012200212068FFF7A2FF2E
:104980002268136843F001031360002038BD012240
:1049900004212068FFF796FFF2E70120F6E70120E7
:1049A000F4E70120F2E70120F0E7000090F83C3046
:1049B000012B45D070B4012380F83C30022380F8ED
:1049C0003D3003685A689C681E4E1F4DAB4218BFAD
:1049D000B34203D122F470024D682A4322F07002E0
:1049E0000D682A435A600368164AB3F1804F18BF16
:1049F000934217D0A2F57C42934213D002F5806215
:104A000093420FD002F5806293420BD002F57842B8
:104A1000934207D0A2F56C42934203D002F5943240
:104A2000934204D124F080048A6814439C600123DB
:104A300080F83D30002380F83C30184670BC704749
:104A40000220704700000140000401407047704799
:104A500070470000026852E8003F23F4907342E878
:104A600000310029F6D1026802F1080353E8001F63
:104A70000D4B0B40083242E800310029F3D1C36EE0
:104A8000012B06D02023C0F88C300023C366436777
:104A90007047026852E8003F23F0100342E80031FB
:104AA0000029F6D1EEE700BFFEFFFFEF704708B523
:104AB000026852E8003F23F0400342E80031002939
:104AC000F6D12023C0F8883000238367FFF7EEFF7C
:104AD00008BD704708B5806B0023A0F85E30A0F8D1
:104AE0005630FFF7F6FF08BD7047000070B504466A
:104AF0000168CB6908688D6840F60F021A4008D13A
:104B000013F0200F05D010F0200F34D115F0805F86
:104B100031D12AB18B4A2A4033D18B4E304230D129
:104B2000E26E012A00F0C68013F4801F03D015F452
:104B3000800F40F09B8113F0800F07D010F0800FA2
:104B400040F09B8115F4000F40F0978113F0400F67
:104B500003D010F0400F40F0978113F4000F03D002
:104B600010F0804F40F0948113F0807F02D0002835
:104B7000C0F2928170BD636F002BFBD02046984736
:104B8000F8E713F0010F09D010F4807F06D001265A
:104B90000E62D4F890103143C4F8901013F0020F55
:104BA0000BD015F0010F08D0216802260E62D4F850
:104BB000901041F00401C4F8901013F0040F0BD0D2
:104BC00015F0010F08D0216804260E62D4F8901069
:104BD00041F00201C4F8901013F0080F0BD010F050
:104BE000200F00D13AB1226808211162D4F8902038
:104BF0000A43C4F8902013F4006F0CD010F0806FBB
:104C000009D022684FF400611162D4F8902042F07C
:104C10002002C4F89020D4F89020002AAAD013F0E3
:104C2000200F09D010F0200F02D115F0805F03D0C3
:104C3000636F0BB120469847D4F8902023689B6897
:104C400013F0400F02D112F0280F2CD02046FFF7AE
:104C500001FF23689B6813F0400F20D0226802F107
:104C6000080353E8003F23F04003083242E80031D4
:104C70000029F3D1D4F880306BB1344A1A65D4F8E6
:104C80008000FDF761FB00283FF474AFD4F880008A
:104C9000036D98476EE72046FFF71BFF6AE7204643
:104CA000FFF717FF66E72046FFF713FF0023C4F85E
:104CB00090305FE713F0100F3FF436AF10F0100F95
:104CC0003FF432AF10230B6223689B6813F0400F50
:104CD00000F09280D4F8802013681D481D498B4253
:104CE00018BF834238D018318B4235D018318B42EF
:104CF00032D018318B422FD018318B422CD0183142
:104D00008B4229D018318B4226D001F556718B4247
:104D100022D018318B421FD018318B421CD0183151
:104D20008B4219D018318B4216D018318B4213D0D8
:104D300018318B4210D018318B420DD05B689BB27A
:104D40000CE000BF0100001020010004D54A00085B
:104D500010000240280002405B689BB2002B3FF429
:104D600009AFB4F85C1099427FF604AFA4F85E3046
:104D7000D369B3F5807F32D0226852E8003F23F434
:104D8000807342E800310029F6D1226802F108035D
:104D900053E8003F23F00103083242E800310029C4
:104DA000F3D1226802F1080353E8003F23F04003E7
:104DB000083242E800310029F3D12023C4F88C30B6
:104DC0000023E366226852E8003F23F0100342E824
:104DD00000310029F6D1D4F88000FDF715F902233F
:104DE0002367B4F85C10B4F85E309BB2C91A89B27C
:104DF0002046FFF779FEBDE6B4F85C10B4F85E30EB
:104E00009BB2C91A89B2B4F85E309BB2002B3FF452
:104E1000B1AE00293FF4AEAE226852E8003F23F461
:104E2000907342E800300028F6D1226802F10803AE
:104E300053E8000F1A4B0340083242E800300028C4
:104E4000F3D12023C4F88C300023E3666367226823
:104E500052E8003F23F0100342E800300028F6D16A
:104E6000022323672046FFF73FFE83E64FF48013BB
:104E70000B62204600F07CFD7CE6A36F002B3FF424
:104E800079AE2046984775E62046FFF710FE71E69A
:104E9000204600F06FFD6DE6204600F06AFD69E6F1
:104EA000FEFFFFEF70B586B00446016883680269B3
:104EB000134342691343C26913430868884A024096
:104EC00013430B602268536823F44053E1680B439B
:104ED0005360A1692268834B9A4201D0236A194327
:104EE0009068814B03400B4393602268D36A23F0A0
:104EF0000F03616A0B43D36222687C4B9A4221D034
:104F00007B4B9A4200F08C807A4B9A4200F0A28050
:104F1000794B9A4200F0B580784B9A4200F0C880F5
:104F2000774B9A4200F0F480764B9A4200F0198158
:104F3000754B9A4200F02C816A4B9A4200F03F81F7
:104F4000802333E0714B5B6D03F03803282B65D869
:104F5000DFE813F02900640064006400640064006A
:104F6000640064004D016400640064006400640037
:104F7000640064002B00640064006400640064004A
:104F8000640064005E006400640064006400640007
:104F900064006400600064006400640064006400F5
:104FA000640064006200012300E008234D498A4246
:104FB00000F02F81E069B0F5004F00F0AF81202BA9
:104FC00000F20782202B00F25182DFE813F01E026C
:104FD00024024F024F0227024F024F024F022C02BF
:104FE0004F024F024F024F024F024F024F02310257
:104FF0004F024F024F024F024F024F024F024F0229
:105000004F024F024F024F024F024F024F023D022A
:105010001023CBE72023C9E74023C7E78023C5E758
:105020003A4B5B6D03F00703052B11D8DFE813F053
:105030000600E10008000A000C000E000023B5E79E
:105040000823B3E71023B1E72023AFE74023ADE700
:105050008023ABE72D4B5B6D03F00703052B0ED8C8
:10506000DFE803F003C90507090B00239EE70823C7
:105070009CE710239AE7202398E7402396E78023B4
:1050800094E7224B5B6D03F00703052B0ED8DFE896
:1050900003F003B40507090B002387E7082385E71E
:1050A000102383E7202381E740237FE780237DE7E8
:1050B000164B5B6D03F00703052B0ED8DFE803F0FA
:1050C000039F0507090B002370E708236EE71023F1
:1050D0006CE720236AE7402368E7802366E700BF88
:1050E000F369FFCF000C0058FFF4FF1100100140DE
:1050F0000044004000480040004C00400050004088
:105100000014014000780040007C00400044025838
:105110007D4B5B6D03F03803282B20D8DFE803F0CC
:10512000151F1F1F1F1F1F1F711F1F1F1F1F1F1F47
:10513000171F1F1F1F1F1F1F191F1F1F1F1F1F1F8D
:105140001B1F1F1F1F1F1F1F1D0001232EE70823EA
:105150002CE710232AE7202328E7402326E7802393
:1051600024E7694B5B6D03F00703052B0ED8DFE8DE
:1051700003F0034A0507090B002317E7082315E787
:10518000102313E7202311E740230FE780230DE7C7
:105190005D4B5B6D03F00703052B0ED8DFE803F0D2
:1051A00003350507090B002300E70823FEE610235B
:1051B000FCE62023FAE64023F8E68023F6E603F532
:1051C0000E339B6D03F00703052B0ED8DFE803F0C9
:1051D000031F0507090B0223E8E60823E6E6102370
:1051E000E4E62023E2E64023E0E68023DEE6042333
:1051F000DCE60423DAE60423D8E60423D6E6042317
:10520000D4E60423D2E60423D0E60423CEE6042326
:10521000CCE6202B27D8022BC0F01A81023B1E2B94
:1052200000F21881DFE813F0500016015600160155
:10523000160116015B001601160116011601160172
:10524000160116016000160116011601160116015D
:105250001601160116011601160116011601160196
:10526000160116016C00402B2CD14FF40040626AED
:10527000264B33F81220B0FBF2F3656805EB4501CD
:10528000994200F2E980B3EB053F00F2E780002687
:1052900033463146FBF7B2FA090241EA10610002D7
:1052A0006B08C0182A46334641F10001FBF7A6FA05
:1052B000A0F54072164B9A4200F2D2802368D86063
:1052C0003046D4E00120D2E0FEF70CFF0028CED11A
:1052D0000020CCE003A8FEF717FF0498F6E7684625
:1052E000FFF72CF80198F1E7074B1B6813F0200F2C
:1052F00008D0054B1B68C3F3C1030648D840E5E757
:105300000548B4E70348B2E7004402589CBB0008D4
:10531000FFFC0F000090D00300093D00202B15D8A2
:10532000202B00F29F80DFE803F031379D9D3A9DEE
:105330009D9D3F9D9D9D9D9D9D9D449D9D9D9D9D54
:105340009D9D9D9D9D9D9D9D9D9D5000402B1BD194
:10535000626A4D4B33F81230B0FBF3F062685308C9
:1053600003EB4000B0FBF2F0A0F110024FF6EF7338
:105370009A4279D883B223F00F03C0F34200184356
:105380002368D860002072E0012070E0FEF734F856
:105390000028DDD100206AE0FEF740F8F8E703A816
:1053A000FEF7B2FE0498F3E76846FEF7C7FF0198E0
:1053B000EEE7364B1B6813F0200F08D0334B1B6809
:1053C000C3F3C1033248D840E2E73248C0E730486F
:1053D000BEE7402B17D14FF40040626A2A4B33F8E6
:1053E0001230B0FBF3F0636800EB5300B0FBF3F056
:1053F000A0F110024FF6EF739A4242D8236880B2B0
:10540000D860002033E0012031E0FDF7F5FF0028EF
:10541000E3D100202BE0FEF701F8F8E703A8FEF740
:1054200073FE0498F3E76846FEF788FF0198EEE7FD
:10543000164B1B6813F0200F08D0144B1B68C3F3E6
:10544000C1031348D840E2E71248C6E71048C4E752
:1054500001200CE001200AE0012008E0012006E024
:10546000012004E0012002E0012000E001200123EE
:10547000A4F86A30A4F8683000236367A36706B015
:1054800070BD0120F3E700BF9CBB00080044025838
:105490000090D00300093D00836A13F0080F06D086
:1054A0000268536823F40043816B0B435360836AA3
:1054B00013F0010F06D00268536823F40033C16A69
:1054C0000B435360836A13F0020F06D002685368DF
:1054D00023F48033016B0B435360836A13F0040F92
:1054E00006D00268536823F48023416B0B4353605A
:1054F000836A13F0100F06D00268936823F4805378
:10550000C16B0B439360836A13F0200F06D00268CF
:10551000936823F40053016C0B439360836A13F088
:10552000400F0AD00268536823F48013416C0B4388
:105530005360436CB3F5801F0BD0836A13F0800F68
:1055400006D00268536823F40023C16C0B435360F8
:1055500070470268536823F4C003816C0B435360A7
:10556000EBE72DE9F84305460E4617469946DDF868
:1055700020802C68E46936EA04030CBF4FF0010C6C
:105580004FF0000CBC453AD1B8F1FF3FF1D0FCF729
:10559000C5FCA0EB0900404534D8B8F1000F33D06A
:1055A0002B681A6812F0040FE3D0B6F1400218BF5E
:1055B0000122802EDDD0002ADBD0DA6912F0080F3C
:1055C00011D1DA6912F4006FD3D04FF400621A627D
:1055D0002846FFF73FFA2023C5F89030002385F8CE
:1055E000843003200CE008241C622846FFF732FABE
:1055F000C5F89040002385F88430012000E00020A9
:10560000BDE8F8830320FBE70320F9E72DE9F0412B
:1056100082B01E46D0F88830202B5BD104460D4660
:105620009046002A18BF002901D1012053E0002331
:10563000C0F890302123C0F88830FCF76FFC074693
:10564000A4F85480A4F85680A368B3F5805F02D014
:105650004FF0000816E0236943B34FF0000811E053
:105660002023C4F88830032035E038F8023B226854
:10567000C3F308039362B4F8562092B2013A92B28F
:10568000A4F85620B4F856309BB293B100963B462E
:10569000002280212046FFF764FF0028E0D1002D82
:1056A000E3D015F8012B23689A62E4E7A8460025A9
:1056B000E8E700963B46002240212046FFF751FFD5
:1056C00018B92023C4F8883005E02023C4F88830B6
:1056D000032000E0022002B0BDE8F0812DE9F04394
:1056E00083B01E46D0F88C30202B7ED104460D4668
:1056F0009046002A18BF002901D1012076E000233E
:10570000C0F890302222C0F88C20C366FCF706FC5B
:105710000746A4F85C80A4F85E80A368B3F5805FB8
:1057200006D0A3B9226972B9FF22A4F8602014E060
:10573000226922B940F2FF12A4F860200DE0FF2296
:10574000A4F8602009E07F22A4F8602005E0B3F10E
:10575000805F0AD00022A4F86020B4F86080B3F51E
:10576000805F0CD04FF0000924E022691AB97F2233
:10577000A4F86020F1E73F22A4F86020EDE7236958
:1057800013B14FF0000915E0A946002512E02023CF
:10579000C4F88C30032029E023685A6A5FFA88F342
:1057A000134005F8013BB4F85E2092B2013A92B280
:1057B000A4F85E20B4F85E309BB28BB100963B46F5
:1057C000002220212046FFF7CCFE0028DFD1002D4B
:1057D000E2D123685B6A08EA030329F8023BE2E7A7
:1057E0002023C4F88C30002000E0022003B0BDE884
:1057F000F08330B583B004460023C0F89030FCF746
:105800008DFB05462268126812F0080F10D123683C
:105810001B6813F0040F28D12023C4F88830C4F883
:105820008C300020E066206784F8840003B030BD2F
:105830006FF07E430093034600224FF40011204690
:10584000FFF78FFE0028E2D0226852E8003F23F0E5
:10585000800342E800310029F6D12023C4F88830C3
:10586000002384F884300320E0E76FF07E43009348
:105870002B4600224FF480012046FFF772FE0028DD
:10588000CAD0226852E8003F23F4907342E8003106
:105890000029F6D1226802F1080353E8003F23F003
:1058A0000103083242E800310029F3D12023C4F873
:1058B0008C30002384F884300320B7E778B310B528
:1058C0000446D0F888300BB32423C4F8883022680B
:1058D000136823F001031360A36AE3B92046FFF7BE
:1058E000E1FA012811D02268536823F490435360F1
:1058F0002268936823F02A0393602268136843F0B8
:10590000010313602046FFF774FF10BD80F8843058
:10591000FCF724FAD8E72046FFF7BEFDDEE70120BA
:1059200070470000436E2BB90123A0F86A30A0F83D
:105930006830704730B403689A68C2F3426299686D
:10594000490F094D6B5C1B01084C615C93FBF1F343
:10595000A0F86A30AB5C1B01A25C93FBF2F3A0F8E9
:10596000683030BC704700BFBCBB0008B4BB000847
:1059700070477047704790F88430012B18D001238E
:1059800080F884302423C0F8883003681A681968C6
:1059900021F00101196022F00052002343660168E2
:1059A0000A602022C0F8882080F8843018467047AA
:1059B0000220704738B590F88430012B1DD0044682
:1059C000012380F884302423C0F8883003681D68E0
:1059D0001A6822F001021A600268936823F060439B
:1059E00019439160FFF79EFF23681D602023C4F8D0
:1059F0008830002084F8840038BD0220FCE738B5E8
:105A000090F88430012B1DD00446012380F88430A7
:105A10002423C0F8883003681D681A6822F0010248
:105A20001A600268936823F0606319439160FFF77E
:105A300079FF23681D602023C4F88830002084F893
:105A4000840038BD0220FCE7014B1868704700BF96
:105A50001000002470B50D4E0D4D761BB61006D00B
:105A6000002455F8043B01349847A642F9D1094E69
:105A7000094D761B06F06CF8B61006D0002455F8D8
:105A8000043B01349847A642F9D170BDC8BF000855
:105A9000C8BF0008D0BF0008C8BF0008830730B5E2
:105AA00048D0541E002A3FD0CAB2034601E0013C50
:105AB0003AD303F8012B9D07F9D1032C2DD9CDB290
:105AC00045EA05250F2C45EA054536D9A4F1100213
:105AD00022F00F0C03F1200EE6444FEA121C03F1F2
:105AE000100242E9045542E9025510327245F8D1DC
:105AF0000CF1010214F00C0F03EB021204F00F0C76
:105B000013D0ACF1040323F003030433134442F82D
:105B1000045B9342FBD10CF003042CB1CAB21C44C9
:105B200003F8012B9C42FBD130BD64461346002C88
:105B3000F4D1F9E703461446BFE71A46A446E0E766
:105B40000FB400B5074983B004AB086853F8042BC1
:105B50008168019300F0E0F803B05DF804EB04B055
:105B6000704700BF100000242DE9F043694CD4F8C1
:105B7000008083B004460E4617461D46B8F1000F5C
:105B800003D0D8F83830002B77D0022F05D0012F62
:105B900000F2AC80002DC0F2A980636EDA0752D506
:105BA0002146404602F062FF216B41B104F14003FF
:105BB000994202D0404603F085F800232363B4F9EC
:105BC0000CC000231CF0800FA361636064D12CF42F
:105BD0004A6C2CF0030C022FA4F80CC06AD001AB65
:105BE0006A462146404603F013FAA3891843A08170
:105BF000002D2FD0002E2ED0D8F83830002B38D0E2
:105C0000009B2660AB42B4F90C301CBF43F4006328
:105C1000A381012F04BF43F00103A3819AB213F0C3
:105C20000803C4E904652CD0D1075DD56D42A56198
:105C3000656E002315F00105A36027D000252846D6
:105C400003B0BDE8F083A3899B05A9D4A06D03F040
:105C50006BF9A5E7009D284603F00AFA06460028DE
:105C600047D0A38943F08003A381D8F83830002BB4
:105C7000C6D1404602F02EFFC2E7404602F02AFF9E
:105C800083E7A360656E15F00105D7D1930524D590
:105C9000284603B0BDE8F0832169404603F012F8BE
:105CA000B4F90CC02CF44A6C2CF0030C022FA4F8AD
:105CB0000CC094D10025002204F14303A26001220C
:105CC000C4E904322360636E4CF0020CD807A4F8D8
:105CD0000CC0DDD41CF4007FDAD1A06D03F026F9EE
:105CE000284603B0BDE8F083A560CBE74FF0FF3551
:105CF000CEE7DDF80090A94504D0484603F0B8F996
:105D0000064620B9B4F90CC04FF0FF35D3E74D4635
:105D1000A7E700BF100000242DE9F04FD5B01C46C6
:105D2000079191460546099003F0F6F8026817922C
:105D300010460E94FAF7E4FF16901DB1AB6B002BE2
:105D400000F02A82079A536EDD0740F13881B2F9DC
:105D50000C2091B28F0409D4079B42F400529A811F
:105D600091B21A465B6E23F4005353660E0740F15E
:105D7000CB80079B1B69002B00F0C68001F01A0343
:105D80000A2B00F0CF8000242BAB4D46CDE92944EF
:105D9000CDE91944CDE91B441294289398461894F0
:105DA00000230B940024CDE914342B78002B00F051
:105DB0009D81AA4604E01AF8013F002B00F0C7803D
:105DC000252BF8D1BAEB050640F0C5809AF80030D3
:105DD000002B00F08B8100234FF0FF329AF8016016
:105DE0008DF883300A930AF1010A08921F462B248A
:105DF0004FF020090AF1010AA6F120035A2B00F204
:105E0000ED80DFE813F0EB02EB00EB00E602EB00C5
:105E1000EB00EB006A00EB00EB005C028002EB00A1
:105E200067028A02EB0085025B005B005B005B009F
:105E30005B005B005B005B005B00EB00EB00EB00DA
:105E4000EB00EB00EB00EB007A01EB00F801D20174
:105E50007A017A017A01EB00EB00EB00EB00E10242
:105E6000EB00EB002D02EB00EB00EB000202EB007D
:105E7000A402EB00EB008307EB00EB00EB00EB0070
:105E8000EB00EB00EB00EB007A01EB00F801D40132
:105E90007A017A017A01C702D401CD01EB00D40264
:105EA000EB006C022F02B502CD01EB0002027E0076
:105EB0008007EB00EB006107EB007E00A6F13003EA
:105EC00000221AF8016B02EB820203EB4202A6F1F8
:105ED0003003092BF5D90A928EE7DDF824B0584635
:105EE00003F01AF843681B931846FAF709FF1C9051
:105EF0000646584603F010F883681993002E40F0C8
:105F0000CD869AF8006075E7079D0998294601F04B
:105F1000ADFC002841F01C83A98901F01A030A2B6B
:105F20007FF431AF079AB2F90E30002BFFF62BAF9A
:105F3000536ED80702D4890541F13B81079909982E
:105F400023464A4655B0BDE8F04F01F04FBCBAEBCE
:105F5000050600F0CB802A9B33442A93299B01330A
:105F6000072BC8E90056299305DC08F108080B9BAC
:105F700033440B932AE70799099828AA03F0E4FF12
:105F800080B90DF1AC08F2E70799099828AA03F047
:105F9000DBFF002800F09B800D9B1BB10998194680
:105FA00002F090FE079A536ED90740F1EA80938978
:105FB0005B0601F1D9820B9855B0BDE8F08F079BC5
:105FC000B3F90C20900591B23FF5C4AE1D46986D13
:105FD00002F0AAFFB5F90C2091B2BBE6002E00F04A
:105FE000858000228DF8EC608DF883200123CDE9B7
:105FF0000C32069308920F92139210923BAD17F059
:10600000020302D006990231069117F0840B07D1E2
:106010000A990698A1EB0009B9F1000F00F370830B
:106020002A9C8AB1299A0DF1830101320134C8F802
:106030000010072A4FF001012A942992C8F8041091
:1060400000F3B68308F1080883B1299B21AA013324
:106050000234C8F80020072B4FF002022A9429933B
:10606000C8F8042000F3B28308F10808BBF1800FE0
:1060700000F06982089B0C9AA3EB020BBBF1000FA6
:1060800000F3AA82FB0500F100820C9BC8F80430E3
:106090001C44299BC8F800500133072B2A942993EC
:1060A00000F3228308F10808780705D50A9B069AB1
:1060B0009D1A002D00F39683DDE90A2306998A4292
:1060C000ACBF9B185B180B93002C7FF45DAF0023D3
:1060D00029930D9B1BB10D99099802F0F3FD0DF169
:1060E000AC0855462B78002B7FF463AE2A9B002B1F
:1060F00041F0D3810023299354E70E9B073323F00B
:106100000702F2E80234CDE91434DDE9143424F056
:1061100000440E92994618462146B54B4FF0FF3287
:10612000FBF7B2FA002840F0EF84B14B4846214615
:106130004FF0FF32FBF78AFA002840F0E584DDE9F2
:10614000140100220023FBF777FA002840F067874C
:106150009DF88320A74DA84B27F080070321472EE9
:10616000C8BF1D4600230D9306910C9108930F9311
:1061700013931093002A3FF442AF069B013306931A
:106180003DE7079B9B899A053FF512AF079CA06DE1
:1061900002F0CCFEA3890BE7099802F09BFCD1E545
:1061A0009AF8006047F0200724E647F01007BA0687
:1061B0000E9B40F13B84073323F007031A465B68CC
:1061C00052F8084B0E929946002BC0F24C84089B63
:1061D000013300F0D88254EA090327F0800B40F025
:1061E000D382089B002B40F0D4825F4600230893A3
:1061F0000C9354AD1DE10E9B002253F8041B8DF847
:1062000083208DF8EC100E93F0E60E9C089B54F85A
:10621000045B4FF000098DF88390002D00F093850A
:106220005A1C00F051861A4649462846FAF768FC7F
:106230000D90002801F00E810D9BCDF820905B1B86
:106240000C930E9423EAE3739DF883200693CDF814
:106250003490CDF83C90CDF84C90CDF8409089E743
:1062600047F0100717F0200900F0D2830E9B073388
:1062700023F00703D3F8049053F8084B0E9327F448
:10628000806B002300228DF88320089A511C00F0B7
:10629000B88054EA09012BF0800740F0B180002A51
:1062A00040F0F685002BA1D11BF001030C9300F008
:1062B000148430238DF84F310DF24F15B9E00E9B49
:1062C00053F8042B0A92002A80F2DA830A9A0E937A
:1062D00052420A929AF8006047F004078AE5BD0628
:1062E00000F1D184FC0600F1D885780600F1A5867E
:1062F000B90540F1D2850E9B0B9953F8042B0E93F0
:1063000011705546EEE69AF800608DF8834071E50D
:106310009AF8006047F080076CE5524612F8016B6E
:106320002A2E01F03F82A6F13003092B924698BF36
:10633000002201F2BC801AF8016B02EB820203EB2F
:106340004202A6F13003092BF5D9089254E547F033
:10635000100B1BF0200900F076830E9B073323F00F
:106360000703D3F8049053F8084B0E93012389E7F1
:106370000E9B53F8044B0E93302378268DF884300F
:106380001E4B189347F0020B8DF885604FF0000903
:10639000022377E79AF80060682E03BF9AF801603D
:1063A00047F400770AF1010A47F0400722E59AF81E
:1063B00000606C2E03BF9AF8016047F020070AF1D5
:1063C000010A47F0100715E59AF8006047F0080742
:1063D00010E59AF8006047F001070BE59DF883305F
:1063E000002B7FF48EAD9AF800608DF8839001E564
:1063F000FFFFEF7FC8BB0008CCBB0008D8BB00087C
:10640000BB46012B00F0C081022B54AD20D1189A5D
:1064100004F00F032409D35C05F8013D44EA097434
:106420004FEA191954EA0903F2D154AB5B1B5F46DA
:106430000C9308990C989DF8832081424FF000033B
:10644000B8BF01460D9306910F931393109391E6F5
:1064500004F00703E40844EA49744FEAD9093033E9
:1064600054EA09012A4605F8013DF1D11BF0010F5C
:10647000DBD0302BD9D03023023A05F8013C54ABA5
:106480009B1A5F460C931546D3E7652E40F3E680D2
:10649000DDE9140100220023FBF7C4F8002800F016
:1064A000DC81299BBF4AC8F8002001330134012256
:1064B000072B2A942993C8F8042000F3CC8408F110
:1064C0000808229B129A934280F2D682169B179A52
:1064D0001C44C8E90023299B2A940133072B2993E4
:1064E00000F3248408F10808129B5D1E002D7FF73D
:1064F000DBAD102D299BDFF8B09240F3BD844946F7
:106500002246B946DDF824B0079C10260F4605E068
:1065100008F10808103D102D40F3AA840133103211
:10652000072BC8E90076CDE92932F1DD28AA2146FA
:10653000584603F009FD00287FF42EADDDE929322D
:106540000DF1AC08E6E70A9B069AA3EB020BBBF140
:10655000000F7FF78FADBBF1100F299ADFF848923B
:106560002CDD1D9621464E46079CDDF82490102315
:1065700006E0ABF1100BBBF1100F08F108081ADDB3
:1065800001321031072AC8E90063CDE92921F0DD85
:1065900028AA214648460DF1AC0803F0D5FC002896
:1065A0007FF4FAACABF1100BBBF1100FDDE9292140
:1065B0004FF01003E4DCB1461D9E0C4601325C44F2
:1065C000072ACDE92924C8F80090C8F804B000F3E0
:1065D000A08308F108084DE5BBF1100F299ADFF8F8
:1065E000C8912DDD41462046A8464C46079DDDF862
:1065F0002490102306E0ABF1100BBBF1100F01F15A
:10660000080119DD01321030072AC1E90043CDE944
:106610002920F0DD28AA2946484603F095FC0028E9
:106620007FF4BAACABF1100BBBF1100FDDE9292000
:106630002BA94FF01003E5DC4546A14688460446E9
:1066400001325C44072ACDE92924C8F80090C8F833
:1066500004B000F3D08108F1080813E5129B012B68
:1066600040F38081299EC8F800500136013401238F
:10667000072E2A942996C8F8043000F37C8308F189
:106680000808169B179A01361C44072EC8E90023F8
:10669000CDE9296400F37C8308F10808DDE91401E1
:1066A00000220023FAF7BEFF002840F07881129BF9
:1066B0000136013B01351C44072EC8F800502996CD
:1066C000C8F804302A9400F35D8108F108081A9B89
:1066D000C8F8043001361C44072E24ABCDE92964E8
:1066E000C8F800307FF7DEAC0799099828AA03F0B4
:1066F0002BFC00287FF450AC2A9C0DF1AC08D3E4AD
:10670000B9F1100FDDE929212BDDCDE91D3B1F96E5
:10671000DDF824B04E461024A946079D04E0103E43
:10672000102E08F1080817DD0132204B1031072A1E
:10673000C8E90034CDE92921F1DD28AA29465846C7
:106740000DF1AC0803F000FC00287FF425AC103EEE
:10675000102EDDE92921E7DCDDE91D3B4D46B14680
:106760001F9EC8F80490013209EB0104072A0F4963
:10677000C8F80010CDE9292400F351839DF8832047
:1067800008F108084DE4BB460A2C79F1000380F0BB
:106790000C83303401238DF84F415F460C930DF28A
:1067A0004F1546E608BC00081CBC00080CBC0008DD
:1067B000079909981D9328AA03F0C6FB00287FF4C7
:1067C000EBAB2A9C1D9B0DF1AC083DE407990998A1
:1067D00028AA03F0B9FB00287FF4DEAB2A9C0DF158
:1067E000AC0843E4102D299B21DD099FDDF81C90A6
:1067F000102604E0103D102D08F1080817DD0133C4
:10680000BB4A1034072BC8E90026CDE92934F1DD55
:1068100028AA494638460DF1AC0803F095FB00283C
:106820007FF4BAAB103D102DDDE92934E7DC0133EC
:10683000AF4AC8F804502C44072BCDE92934C8F8D6
:1068400000207FF739AC0799099828AA03F07CFB50
:1068500000287FF4A1AB2A9C2EE42299002940F362
:106860001481DDF84090129B9945A8BF9946B9F173
:10687000000F0BDD299B01334C44072BC8E900595D
:106880002A94299300F39A8508F10808109EB9F11B
:10689000000FA8BFA6EB0906002E00F34683DDF823
:1068A00040B07905AB4400F1CE84229B129A93420A
:1068B00002DBFA0740F1B883169A17991444C8E925
:1068C0000012299A2A940132072A299200F383851B
:1068D00008F10808129AAE18A6EB0B06D51AAE42BC
:1068E000A8BF2E46002E0DDD299BC8F800B001334D
:1068F0003444072BC8F804602A94299300F3F185E7
:1069000008F10808002EA8BFAD1B002D7FF7CCAB07
:10691000102D299BDFF8DC9140F3AE8249462246D8
:10692000B946DDF824B0079C10260F4605E008F1B3
:106930000808103D102D40F39B8201331032072BC5
:10694000C8E90076CDE92932F1DD28AA214658466A
:1069500003F0FAFA00287FF41FABDDE929320DF1CC
:10696000AC08E6E7FE073FF57DAE299EC8F800506B
:10697000013601340123072E2A942996C8F80430E1
:106980007FF7A3AE0799099828AA03F0DDFA00283B
:106990007FF402ABDDE929640DF1AC0897E6129BA8
:1069A0005D1E002D7FF793AE102DDFF8489140F368
:1069B0007F8222460897099C079F4FF0100B05E045
:1069C00008F10808103D102D40F370820136103296
:1069D000072EC8E9009BCDE92962F1DD28AA3946D6
:1069E000204603F0B1FA00287FF4D6AADDE9296237
:1069F0000DF1AC08E6E70799099828AA03F0A4FA74
:106A000000287FF4C9AA2A9C0DF1AC08FFF73ABB15
:106A100017F0100372D117F0400200F0BD820E9AF9
:106A200052F8044B0E929946A4B228E453F8044B52
:106A30000E93FB0656D47D0651D544F3C0394B4620
:106A400024B2FFF7C1BB1BF0100340F036811BF0EE
:106A5000400200F092820E9A52F8044B0E92994630
:106A6000A4B201230EE42D2364428DF8833069EB38
:106A70004909BB46012308E4F8077FF515AB25E576
:106A80009AF800600E93FFF7B5B9299B1A4AC8F827
:106A90000020013301340122072B2A942993C8F8DE
:106AA000042000F3708408F10808002940F01E82D9
:106AB000129A07F0010313433FF4F6AA169B1799A5
:106AC000E218C8E90013299B2A920133072B299366
:106AD00000F3618308F1080819E254ADA9E4B80590
:106AE00000F1B4824FEAE4794B46FFF76DBB00BF7B
:106AF0000CBC00081CBC000808BC00080E9B53F826
:106B0000044B0E93FFF7BBBBDDE9140102460B46B5
:106B1000FAF7BAFD002840F0A085612E00F05085FC
:106B2000412E00F09982089B013326F02003069342
:106B300000F08F85472B00F07985DDE9141247F4CA
:106B400080730F931346002BC0F2ED850C93002346
:106B50001D938B460D93069B462B00F04A84452BD4
:106B600000F04F850899019126A9049123A903916A
:106B700022A9029102210C9B099800915A4600F02B
:106B800083FF069B472B054640F01C8617F0010F3C
:106B9000B9460F9F40F0D984269B5B1B1293069B3E
:106BA000472B00F01883069B462B00F05F84229B46
:106BB0001093109B069A013B412A229300F0AA856C
:106BC000F2B20021002BB8BF109B8DF89020BABF05
:106BD000C3F101032D222B22092B8DF8912040F3C4
:106BE00063850DF19F04BD4F2246104687FB0321AC
:106BF000DA17C2EBA10202EB8201A3EB41013031B3
:106C000000F8011C19466329134600F1FF32ECDC41
:106C10003033D9B2831E9C4202F8011C40F2CE856B
:106C200013460DF1920201E013F8011B02F8011B5B
:106C30009C42F9D10DF1A1030DF192021B1A1344EC
:106C400024AA9B1A1A93129B1A9A012B1A440C928B
:106C500040F372850C9B169A13440C930C9A0023F4
:106C600029F4806722EAE27247F480770F93069254
:106C7000139310931D9B002B40F0DE829DF8832020
:106C80000893FFF777BA0E9B0B9853F8041B0E93EB
:106C9000C217C1E900025546FFF724BA199B002B21
:106CA0003FF42FA9199B1B78002B3FF42AA99AF8CF
:106CB000006047F48067FFF79DB80E9B53F8044BC4
:106CC0000E930123FFF7DEBA854B189317F02009C6
:106CD00049D00E9B073323F00703D3F8049053F8F1
:106CE000084B0E93F80709D554EA090306D0302360
:106CF0008DF8856047F002078DF8843027F4806BAB
:106D00000223FFF7BFBABB46FFF723BB754B1893AF
:106D1000DCE70799099828AA03F016F900287FF400
:106D20003BA92A9C0DF1AC08FFF7A4B90799099873
:106D300028AA03F009F900287FF42EA92A9C0DF156
:106D4000AC08FFF7D1BB062B294628BF06230895C0
:106D50000D952A460693644D0E940C930F91139152
:106D60001091FFF707BA17F0100369D00E9B53F884
:106D7000044B0E93B6E70799099828AA03F0E4F8A4
:106D800000287FF409A9DDE929640DF1AC0878E455
:106D90000799099828AA03F0D7F800287FF4FCA8DF
:106DA000DDE929640DF1AC0878E40BF4806300227E
:106DB000CDE90CA80696DDF8648054AF16469A46D5
:106DC0000CE00023204649460A22F9F717FD0A2C59
:106DD00079F100031BD3044689462F4620460A2238
:106DE00000234946F9F70AFD30327D1E013607F8C7
:106DF000012CBAF1000FE4D098F800309E42E0D1A7
:106E0000FF2EDED00A2C79F1000380F0F480CDF85B
:106E100064801296DDE90CA8069EFFF706BB079971
:106E200009981D9328AA03F08FF800287FF4B4A8CE
:106E30009DF883202A9C1D9B0DF1AC08FFF7F1B84B
:106E400017F0400200F0B6800E9A52F8044B0E92F2
:106E50009946A4B246E70799099828AA03F074F85E
:106E600000287FF499A82A9C0DF1AC08FFF729BBF4
:106E700014463A464F46914601332C44072BC8F836
:106E80000090C8F80450CDE929347FF70BA92BE412
:106E9000012BBB467FF4B8AA7BE40E9B0B9953F8F9
:106EA000042B554611600E93FFF71CB9089F14463A
:106EB00001362C44072ECDE92964C8F80090C8F8A3
:106EC00004507FF702AC5DE52846CDF820900E9483
:106ED000F9F716FF03460C90FFF7B4B967666666CC
:106EE000D8BB0008ECBB000800BC0008169B179834
:106EF000E218C8E90003299B2A920133072B299342
:106F000000F3498108F108080029C0F2FA821299B9
:106F1000C8F8005001338C18072BCDE92934C8F884
:106F200004107FF7BFA8FFF7DFBB102E299BDFF807
:106F3000C09252DD484642462146A846B946099CC1
:106F4000079D4FF0100B074603E00832103E102E4D
:106F50003DDD01331031072BC2E9007BCDE929313A
:106F6000F3DD28AA2946204602F0EEFF00287FF430
:106F700013A8DDE929312BAAE8E70E9B1BF4007961
:106F800014BF53F8044B53F8044B0E931CBF9146A7
:106F9000E4B20123FFF776B90E9B17F4007914BF12
:106FA00053F8044B53F8044B0E931CBF9146E4B2C4
:106FB000FFF765B90E9B17F4007914BF53F8044B23
:106FC00053F8044B0E931CBF9146E4B28AE6454643
:106FD00090463A460C464F46914601333444072BBF
:106FE000CDE92934C8F80090C8F8046000F3E680C1
:106FF00008F1080853E41C9B1B99ED1A1A46284611
:1070000002F034FF98F801300BB108F10108204676
:1070100049460A2200230026F9F7F0FBDBE62D2281
:107020008DF88320FFF796B8129AAE18A6EB0B06E0
:10703000D51AAE42A8BF2E4664E40E9B0B9953F8B6
:10704000042B0E9311805546FFF74CB844F3C0193A
:107050004B4664B2FFF7B8B830238DF8843058231C
:107060008DF88530089B632B47F0020400F39B8268
:1070700000230D933BADDDE9141247F481730F93A8
:107080001346002B2746C0F220820C9326F02003E3
:10709000069300238B461D93612E00F0ED82412E56
:1070A0007FF459AD22AA0C99584602F04FFE0022F7
:1070B0004FF07F53FAF74EF802460B46CDE9102306
:1070C00000220023FAF7AEFA08B101232293494BBC
:1070D0000C93089BCDE912A6CDE91E78DDF830A00F
:1070E000DDE9106703F1FF39AB46109506E0002299
:1070F000002309F1FF39FAF795FAE8B93E4B00226F
:1071000030463946FAF726F80F460646FAF7D2FA1D
:107110000446F9F7B5FF0B46024639463046F9F703
:1071200061FE1AF80430B9F1FF3FD8464D460BF81E
:10713000013B06460F46DAD1304639462F4BDDF883
:1071400048A0139ECDF848800022A946DDF87C8037
:10715000109D1E9FCDE91001FAF78CFA002840F02F
:107160003482DDE91001254B0022FAF75BFA10B1F9
:10717000E10700F12A824B46002B06DB01335B441A
:1071800030220BF8012B5B45FBD1ABEB0503B94675
:1071900012930F9F03E50799099828AA02F0D4FEDD
:1071A00000287EF4F9AEDDE9293222990DF1AC0810
:1071B000AAE6906D01F0BAFEFEF7C0BE07990998E5
:1071C00028AA02F0C1FE00287EF4E6AE2A9C0DF14A
:1071D000AC08FFF764BB229B1093DA1C02DB089A11
:1071E00093420DDD023E26F020030693E1E400BF4A
:1071F0001CBC0008ECBB0008000030400000E03F71
:10720000109B129A9342C0F2568119F0010F00F0C0
:107210008782169A13440C9319F4806F03D0109B45
:10722000002B00F350820C9B23EAE373069367263E
:1072300000230F9313931DE52D2200238DF8832047
:107240000893FEF79ABF129BCDF830A04246DDF8B6
:107250004C801097EB1808935E46199FDDF87090EC
:10726000DDF824A0DDF81CB00F9B13952146B8F182
:10727000000F2ED0002B6BD1013F08F1FF381B9B74
:10728000C2E90039299B01334944072B2A912993EC
:1072900062DC0832089B38789B1B8342A8BF0346F8
:1072A000002B1C460ADD2998013019440728C2E941
:1072B00000632A9129905ADC38780832002CACBF40
:1072C000051B0546002D15DC06440F9BB8F1000F89
:1072D000D0D1002B3CD1DDE91235EB189E42199735
:1072E000B346DDF830A0109F90460C4628BF9B4661
:1072F000FFF7DBBA102D29981DDD102404E0103DA6
:10730000102D02F1080216DD0130AC4B10310728B8
:10731000C2E90034CDE92901F1DD28AA59465046D9
:1073200002F012FE00287EF437AE103D102DDDE98C
:1073300029012BAAE8DC0130A04B5560294407281D
:10734000CDE9290113602CDC387808320644BCE70B
:107350000F9B013B0F9392E728AA5946504602F033
:10736000F3FD00287EF418AE2A992BAA92E728AAEA
:107370005946504602F0E8FD00287EF40DAE3878FC
:107380002A992BAA9AE70799099828AA02F0DCFD06
:1073900000287EF401AE22992A9C0DF1AC08FFF77B
:1073A00084BB28AA5946504602F0CEFD00287EF440
:1073B000F3AD38782A992BAA064486E707990998ED
:1073C00028AA02F0C1FD00287EF4E6AD2A9C0DF14A
:1073D000AC08FFF75BBA0799099828AA02F0B4FD38
:1073E00000287EF4D9AD229B2A9C0DF1AC08FFF752
:1073F00071BA0899019126A9049123A9039122A9A0
:10740000029103210C9B099800915A4600F03CFB25
:107410000378302B054600F09581229B089AB946E7
:1074200013440F9FEC180C99584600220023FAF7DA
:10743000F9F810B12346FFF7B0BB269BA342BFF477
:10744000ACAB30215A1C26921970269B9C42F9D86D
:10745000FFF7A3BB089B9DF883200E9406930C9323
:1074600008900F9013901090FEF784BE229A10920D
:10747000002A40F38181089909F001030B4340F091
:107480005581109B0C93662619F4806F40F01C8187
:107490000C9B23EAE3730693CAE60799099828AA86
:1074A00002F052FD00283EF425AEFEF77BBD00231E
:1074B0000893FEF7A1BC129B169A9A18109B0C9287
:1074C000002B40F34D816726DEE726F0200306936C
:1074D000DDE914349B4604F100430C932D231D93E6
:1074E000DAE50799099828AA02F02EFD00287EF413
:1074F00053AD229D129B2A9C5D1B0DF1AC08FFF73A
:1075000001BA4E421031DFF8B49034DA4146DDF86A
:1075100024B0A8461024079D03E00831103E102E29
:1075200027DD01331032072BC1E90094CDE9293260
:10753000F3DD28AA2946584602F006FD00287EF40D
:107540002BADDDE929322BA9E8E7089BEC186AE7A7
:10755000079B5B6EDD0707D4079B9B899C0503D4C3
:10756000079B986D01F0E2FC4FF0FF330B93FEF7A1
:1075700022BD4546884601333244072BCDE92932E6
:10758000C8F80090C8F804607FF7A4AA0799099882
:1075900028AA02F0D9FC00287EF4FEACDDE92932ED
:1075A0000DF1AC08B3E40998591C01F069FD0546DA
:1075B000002800F00D810D905DE500BF1CBC0008A7
:1075C00030238DF8843078234AE5129B26930C9B58
:1075D0001BF8012CD97B8A425B4609D1302003F885
:1075E000010C269B5A1E269213F8012C9142F6D0CC
:1075F000392A0BBF0C9A0132927AD2B203F8012CCD
:10760000C3E508990C9B09984C1C26A9049123A951
:10761000039122A9029102215A460194009100F09F
:1076200033FA0546B9462C440F9FFCE6089B002B15
:1076300008BF0123089347F480730F93159B002B19
:10764000C0F2AE80DDF850B01D900C930D90FFF7A6
:1076500089BA06230893FFF770BA159B604D002B7B
:10766000B4BF2D229DF883205E4BB8BF8DF88320D8
:1076700027F08007FEF772BD22AA0C99584602F047
:1076800065FB00224FF07F53F9F764FD02460B467D
:10769000CDE9102300220023F9F7C4FF08B101232C
:1076A0002293514B0C9314E5002962D130228DF8BE
:1076B00092200DF19302303302F8013B24ABD31A30
:1076C0001A93FFF7C0BA672619990B78FF2B7BD066
:1076D0000024109A204603E001300131FF2B08D02E
:1076E000934206DAD21A4B78002BF5D10B7801348D
:1076F000F4E71991109213900F940F9A139B1C9911
:1077000013440C9A01FB03230C9323EAE3730693BF
:10771000FFF7B0BA06F10F02D2B20121FFF752BA59
:10772000109B0C9378E500230D93D1E6169BD3189C
:1077300019440C916626A7E619F0010F3FF48EAAB2
:10774000FFF788BA0C99584600220023F9F76AFF20
:1077500000287FF462AE089BC3F1010322935DE62B
:10776000C3F101031A4422EAE2730C9206936726DE
:107770005EE50DF192029EE7089A09F0010959EAC7
:10778000020304D10123069366260C9350E5169B51
:1077900001331A4422EAE2730C920693662647E507
:1077A0000D9095E60E9B9AF80160924653F8042BD3
:1077B0000E9342EAE2720892FEF71CBB02231A9370
:1077C000FFF741BA089C2DE700230F93139394E72A
:1077D000079A938943F040039381FEF7E3BB00BF10
:1077E000D0BB0008D4BB0008D8BB0008F0B51F46CA
:1077F0008B89ADF26C4D23F00203ADF80C304B6E6B
:107800001993CB89ADF80E30CB6907934B6A099376
:107810001AAB009304934FF4806315460646029317
:10782000059316A800230C46069301F079FB2A461F
:107830003B4669463046FEF76FFA051E07DB694690
:10784000304601F013F9002818BF4FF0FF35BDF89E
:107850000C305B0603D5A38943F04003A38116983F
:1078600001F060FB28460DF26C4DF0BD38B5334B8E
:107870001B6805460C460BB19A6B12B3B4F90C3079
:1078800018079AB225D5216900292DD012F00100E0
:1078900007D00020A06060694042A06139B100209B
:1078A00038BD950758BF6069A0600029F7D112065E
:1078B00058BF0846F4D543F04003A3814FF0FF3092
:1078C00038BD184601F006F9B4F90C3018079AB221
:1078D000D9D4D1062AD5520714D4216943F008031C
:1078E000A3819AB20029D1D102F42070B0F5007FB3
:1078F000CCD02146284601F01BFBB4F90C3021699D
:107900009AB2C3E7216B51B104F14002914204D015
:10791000284601F0D7F9B4F90C300022226321691E
:107920000022C4E9001223F02403D7E7092243F020
:1079300040032A604FF0FF30A38138BD10000024BF
:10794000024B13B1024800F005B870470000000078
:10795000F98B0008002301461A46184603F024BAA2
:107960002DE9F04F03690C69A34283B0C0F2868011
:10797000013C01F11405A30000F11408009355F82F
:10798000243058F8242001338A469A4208EB8401B7
:10799000814605EB84070191B2FBF3F638D300234F
:1079A000AE4640469B465EF8041B02681FFA81FC07
:1079B00006FB0C33090C4FEA134C06FB01CC99B2C1
:1079C000ABEB01011FFA8CF311FA82F1C3EB124207
:1079D00002EB214289B241EA0241774540F8041B9B
:1079E0004FEA1C434FEA224BDDD2009B58F803308C
:1079F00073B9019B043B984504D307E0984504F113
:107A0000FF3403D253F80429002AF7D0C9F81040F4
:107A10005146484602F072F800282BDB01364046FA
:107A2000002355F8041BD0F800C08AB29A1A0B0C38
:107A300012FA8CF2C3EB1C4303EB224392B242EAEC
:107A40000342AF4240F8042B4FEA2343E9D258F8EF
:107A5000242008EB84036AB9043B984504D307E06B
:107A6000984504F1FF3403D253F80429002AF7D0D3
:107A7000C9F81040304603B0BDE8F08F002003B0D5
:107A8000BDE8F08F000000002DE9F04F016C99B0C7
:107A900090469946CDE90489259D044641B1426C42
:107AA0004A60012393408B6001F0CCFD00232364E6
:107AB000B9F1000AB4BF012300232B60764BBCBF91
:107AC0002AF0004ACDF814A033EA0A0300F0AA8095
:107AD000DDE904231046194600220023CDE90A01FE
:107AE000F9F7A0FD074670B1249A01231360269B85
:107AF000002B00F0E48269481860431E039303984A
:107B000019B0BDE8F08F16AB019317AB0093204678
:107B1000DDE90A2302F0B8F85FEA1A56054640F09C
:107B20009780DDE916763E4406F23240202840F385
:107B3000B583C0F140000AFA00FA06F2124028FAB2
:107B400000F04AEA0000F9F78BFA0123013EA1F1A7
:107B5000F8710F93524B0022F9F744F948A3D3E987
:107B60000023F9F7F7FA48A3D3E90023F9F73CF922
:107B7000804630468946F9F783FA45A3D3E90023C6
:107B8000F9F7E8FA02460B4640464946F9F72CF960
:107B900080468946F9F78EFD002283460023404641
:107BA0004946F9F749FD002840F07C82BBF1160FE9
:107BB00000F26B823B4B03EBCB03D3E90023DDE9FF
:107BC0000A01F9F739FD002872D00023BE1B0E937D
:107BD000731E0BF1FF3B069300F15E8200230993B5
:107BE000BBF1000F6BDA099BCDF81CB0A3EB0B03C4
:107BF0000993CBF100030D93229B092B4FF0000B4F
:107C000066D8052B40F34883043B22930026229B31
:107C1000023B032B00F26886DFE813F05C04590492
:107C200050043304249A42F20F73CAF3130A136008
:107C30005AEA08031AD1269B002B00F064861A4BDF
:107C400003930833269A0398136019B0BDE8F08FA8
:107C5000DDE90A12C2F31303084643F07F510F9780
:107C6000A6F2FF36169F41F4401173E7269B002BC6
:107C700040F0EA830D4B039341E700BFAFF3008070
:107C800061436F63A787D23FB3C8608B288AC63F22
:107C9000FB799F501344D33F0000F07F09BC0008DC
:107CA0000000F83F78BD000830BC00082CBC00087C
:107CB000BE1B731E069300F185840E900990069BEF
:107CC0005B44CDE9063B00230D93229B092B98D9F9
:107CD0000023CDE9223301264FF0FF330C960893A1
:107CE000089B129300216164204601F085FC0390FB
:107CF000002800F00186039B2364089B0E2B00F2F2
:107D00001381002E00F010810799002940F35C8454
:107D1000AE4B01F00F0203EBC2034FEA2118C90575
:107D2000D3E9006740F11484A94BDDE90A01D3E9E6
:107D30000823F9F739FBCDE9100108F00F084FF0DF
:107D4000030AB8F1000F13D0DFF8849218F0010F86
:107D500009D030463946D9E90023F9F7FBF90AF191
:107D6000010A06460F465FEA680809F10809EDD1E5
:107D7000DDE9100132463B46F9F716FB804689469D
:107D80000E9B43B1934B002240464946F9F754FC01
:107D9000002840F030855046F9F772F942464B46CC
:107DA000F9F7D8F98C4B0022F9F71EF8A1F15073BE
:107DB000CDE910011193089B002B00F09780079BE1
:107DC0001493089B13930C9B002B00F0A584139A2B
:107DD0007E4B8249039E03EBC20353E9022300203A
:107DE000F9F7E2FADDE91023F8F7FCFFCDE910011D
:107DF00049464046F9F75EFC0746F9F741F9024665
:107E00000B4640464946F8F7EDFF3037DDE91023D1
:107E100006F8017B80468946F9F70EFC002840F001
:107E20002985CDF854B00027DDE910AB1095139DDE
:107E300013942AE00137AF4280F22C85684B5046FC
:107E400059460022F9F786F9654B002282468B4697
:107E500040464946F9F77EF989468046F9F72AFCFB
:107E60000446F9F70DF902460B4640464946F8F735
:107E7000B9FF303406F8014B52465B4680468946CE
:107E8000F9F7DAFB002840F0F38442464B465149AB
:107E90000020F8F7A7FF52465B46F9F7CDFB002814
:107EA000C8D0DDE91343109D039A079302E0964280
:107EB00000F0C884B24616F8013D392BF7D00133E3
:107EC000DBB23370079B01330793C8E15046F9F7E3
:107ED000D7F842464B46F9F73DF93F4B0022F8F7F9
:107EE00083FFA1F15073CDE9100111933D4B404642
:107EF00049460022F8F776FFDDE910894B464246F5
:107F000006460F46F9F7B6FB8146002840F0AA84E2
:107F1000DDE91001024601F1004330463946F9F728
:107F20008BFB002840F04583179B002BC0F28C8010
:107F3000079A0E2A00F38880244B03EBC203D3E98F
:107F400000AB239B002B1BDA089B002B18DC40F0B6
:107F50002E83244B002250465946F9F7FBF802467F
:107F60000B46DDE90A01F9F771FBDDF820904E467A
:107F7000002800F0C782239BDDF80C80DF43C9E2B4
:107F8000DDE90A7852465B4638464146F9F70CFA75
:107F9000F9F790FB81460990F9F772F852465B4673
:107FA000F9F7D8F8039E0B46024641463846F8F7E3
:107FB00019FF09F1300306F8013B089B012B00F083
:107FC0005C830694012704951C462AE078BD0008CE
:107FD00050BD00080000F03F00001C400000E03FE2
:107FE000000024400000144052465B46404649468B
:107FF000F9F7DAF9F9F75EFB0546F9F741F8524669
:108000005B46F9F7A7F801370B460246494640465A
:10801000F8F7E8FE05F13003A74206F8013B00F04F
:108020002983AC4B0022F9F795F800220023804603
:108030008946F9F7F7FA0028D6D0049D069C079BDD
:1080400001330793B2460AE10C9A002A3DD0229AE6
:10805000012A40F39C82089B03F1FF380D9B4345A6
:10806000C0F26D82A3EB0808089B002BC0F23C8392
:10807000069A1A440692099A17461A44099201214F
:10808000204601F087FB064623E00123BE1B0E932A
:10809000731E06937FF5A2ADC6F101030993002379
:1080A00006939DE55846F8F7EBFF42464B46F9F735
:1080B000B9FA00287FF47AAD0BF1FF3B76E5864BE9
:1080C0000393039819B0BDE8F08FDDF83480099F61
:1080D0000C9E002F0CDD069900290B4608DD099A3D
:1080E000B942A8BF3B46D21AFF1ACB1A099206938F
:1080F0000D9BDBB10C9B002B00F05D82B8F1000FF3
:108100000FDD31464246204601F020FC2A4601465A
:108110000646204601F06CFB29460546204601F044
:1081200091FA0D9BB3EB080240F0D8820121204662
:1081300001F030FBBBF1000F814600F3B480229BBD
:10814000012B40F386814FF0000A0120BBF1000FA4
:1081500040F0B580069A104410F01F0000F09380A4
:10816000C0F12003042B40F3D283099BC0F11C0013
:1081700003440244099307440692099B002B05DD42
:1081800029461A46204601F041FC0546069B002B75
:1081900005DD49461A46204601F038FC81460E9B13
:1081A000002B40F03681089B002B40F31D810C9B77
:1081B000002B40F0A080079B01330793DDF80C8073
:1081C000DDF820A0012707E0294600230A222046E7
:1081D00001F042FA0137054649462846FFF7C0FB41
:1081E000574500F1300308F8013BEDDB089A002AFF
:1081F000C8BF9346039AD8BF4FF0010B93440027A2
:10820000294601222046049301F000FC4946054618
:1082100001F074FC002840F3A8811BF8013C039A8C
:108220000BF1FF3B04E05A4500F0AA811BF8013D29
:10823000392B0BF1010AF6D001338BF80030494697
:10824000204601F0FFF956B12FB1B74203D03946AD
:10825000204601F0F7F93146204601F0F3F92946AE
:10826000204601F0EFF900238AF80030249B079A9A
:108270001A60269B002B3FF442AC0398C3F800A081
:1082800019B0BDE8F08F1C20099B03440993069B9D
:1082900003440744069370E70126B8E4C0F12000C8
:1082A00008FA00F04FE401465A46204601F04EFB22
:1082B000229B012B814640F3B3814FF0000AD9F88D
:1082C000103009EB8303186901F016FAC0F12000A1
:1082D00040E700BF0000244008BC000831460023EE
:1082E0000A22204601F0B8F9129B002B064640F303
:1082F000E782CDE90783002F00F31A81BAF1000F5E
:1083000040F0D581B046049B039F089903F0010219
:108310007B1E1944229B0C92134309910A934946F0
:108320002846FFF71DFB31468346284601F0E6FB51
:10833000424649468246204601F000FCC26801469A
:108340000BF13003002A42D106902846089301F031
:10835000D5FB06990490204601F074F9049A089B15
:108360001AB90A99002900F09B82BAF1000FC0F2F5
:10837000638122994AEA010A0C9951EA0A0100F044
:108380005B81002A00F3B481099A3B7007F1010A6E
:108390009742D34600F0B281294600230A222046A4
:1083A00001F05AF94645054631464FF000034FF0BB
:1083B0000A02204612D001F04FF94146064600233A
:1083C0000A22204601F048F957468046A7E7204692
:1083D000049301F037F9049B0122C6E701F03CF950
:1083E0005746064680469AE7229B022B79DC0C9B77
:1083F000002B80D1079B4946013328460793FFF79E
:10840000AFFADDF80CB000F130030BF8013B0027A8
:10841000F6E64946284601F071FB0028BFF6C3AED8
:10842000294600230A22204601F016F9079B03F192
:10843000FF380C9B0546002B7FF450AF129B002B9E
:1084400040F335820893B9E6AF4B03930333FFF74C
:10845000F9BBDDE9041200297FF475AEC2F3130302
:10846000002B7FF470AEA94B1340002B00F0FE816F
:10847000099B01330993069B013306934FF0010AD0
:1084800063E601230C93239B079A13441293013351
:10849000012B1F460893B8BF01270021172F6164E5
:1084A0007FF722AC012204235B0003F11400B842E1
:1084B000114602F10102F7D9616415E401230C931E
:1084C000239B002B4CDD129308931F46E5E7002306
:1084D0000C93D8E700230C93F2E7129BCDF81C8095
:1084E0000893089B002B7FF446AD494605222046A1
:1084F00001F0B2F801468146284601F0FFFA002853
:108500007FF739AD0398079F3123804600F8013B80
:10851000013703904946204601F094F87B1CDDF8B2
:108520000CA00793CDF80C80002E7FF494AE96E655
:1085300031463A46204601F069FA0646DEE60D9BD2
:10854000CDF83480A8EB03039B444FF000088BE583
:10855000DDE90A234FF0020ACDE91023FFF7F1BB52
:10856000012323930893FFF7BBBB03D1049BDB07D5
:108570003FF553AEDA461BF8013D302BFAD05EE6EC
:10858000079B039A013307933123137057E60F9A21
:10859000002A00F0268103F23343069ADDF8348086
:1085A0001A440692099A17461A44099267E54FF051
:1085B00000094E46DFE429460D9A204601F0C6F92F
:1085C0000546B3E50E9067E500F00F81079A504B22
:1085D000564206F00F0203EBC203D3E90023DDE9A4
:1085E0000A01F8F7B7FD36118046894600F071811F
:1085F000484F00234FF0020AF20706D5D7E90023BF
:10860000F8F7A8FD0AF1010A0123761007F108071F
:10861000F2D1002B3FF4B4AB80468946FFF7B0BBE4
:10862000049B002B7FF449AEDDE90412C2F313036F
:10863000002B3FF418AF40E6002A12DD2946012244
:108640002046049301F0E2F94946054601F056FA46
:108650000028049B40F31881392B00F0F9800BF1BE
:108660003103BA460AF8013B079B013337460793AB
:108670004646E4E50995069C049D02460B46F8F73C
:10868000B3FB52465B4680468946F8F7F3FF60B974
:1086900052465B4640464946F8F7C4FF00283FF47F
:1086A000CEAC099BD9077FF5CAAC039A02E4716886
:1086B000204600F0A1FF0746002800F00E81336934
:1086C00002339A0006F10C010C30F8F769FA3946CA
:1086D0000122204601F09AF9804614E629462046F8
:1086E00001F034F9054621E5DDE908239F1AC6E4C7
:1086F000392B00F0AD80BA460133B3E7079A013257
:108700003746079246467BE52CBC00080000F07F08
:1087100078BD000850BD0008DDF84CA0844901EB8D
:10872000CA01DDE9102351E90201F8F713FDCDE993
:10873000100149464046F8F7BDFF0646F8F7A0FC91
:108740000B46024649464046F8F74CFB039F53460A
:108750003036012B07F8016B8046894600F0AE8069
:10876000139E039B1E44734B002240464946F8F774
:10877000F1FC89468046F8F79DFF8246F8F780FCB9
:108780000AF1300A02460B4640464946F8F72AFBF2
:1087900007F801ABB74280468946E4D1664B002218
:1087A000DDE91001F8F720FB42464B46F8F744FF9D
:1087B000002864D1DDE910235F490020F8F712FB9F
:1087C00042464B46F8F756FF00283FF4ADABB246A1
:1087D000013E1AF8013C302BF9D0149B013307936A
:1087E0003DE5169BC3F13603D7E6DDE90A894FF074
:1087F000020AFFF7C5BA089B002B3FF467AB129B38
:10880000002B7FF791AB079A013ACDE9133240462E
:10881000484B00224946F8F79DFC804689460AF1FC
:108820000100F8F72DFC42464B46F8F793FC434B0A
:108830000022F8F7D9FAA1F15073CDE91001119394
:10884000FFF7C1BA079B013307933123FFF739BB09
:10885000079BBB4601330793392337460BF8013B8F
:108860004646DCE44FF000094E464BE69A466CE47F
:10887000109D139C149B01330793B246EFE4149BA5
:10888000039A0793FFF716BB7FF4EBAEDA077FF589
:10889000E8AEE1E6DDF854B0109D139CFFF744BB51
:1088A000392BD5D0BAF1000F3FF7D9AED9E6229BCC
:1088B000022B3FF712AECDF81C809BE53E466DE7DC
:1088C000229B022B3FF709AE129BCDF81C80089328
:1088D00011E54FF0020AFFF753BA194B19483A460F
:1088E00040F2EA2102F0A6FA0026666431462046EC
:1088F00000F082FE039078B9114B124800224FF429
:10890000D57102F097FA104B0393FFF7F8B83FF4D4
:1089100034ACC0F13C00B7E4039B236401224FF068
:10892000FF33239612930C920893FFF7FDBA00BF12
:1089300078BD0008000024400000E03F00001C401B
:108940003CBC000850BC000830BC0008B1F90C2049
:10895000F8B50C461107074642D4636842F400623A
:10896000002BA28159DDA56A002D54D000233E685A
:108970003B6093B212F4805253D1E169012338462F
:10898000A847421C63D0A389A56A5B0705D5636825
:10899000C01A236B0BB1E36BC01AE16902460023D6
:1089A0003846A847411C3ED13B68002B3BD01D2BCD
:1089B00001D0162B52D1A3892269226023F40063CF
:1089C00000216160A381216B3E6021B304F140036B
:1089D000994202D0384600F075F900202063F8BDB6
:1089E0002669C6B193B2256826609A070CBF6369F1
:1089F0000023AD1BA3600CE0D4F824C0E1692B4632
:108A000032463846E047B0F1000CA5EB0C05664451
:108A100016DD002DF0DC0020F8BDE36B002BA2DC9E
:108A2000F9E7206DB1E7B4F90C302269226023F434
:108A30000063A3810022DB046260C4D52065C2E725
:108A4000A38943F040034FF0FF30A381F8BD3B689A
:108A5000002B98D01D2B06D0162B04D0A38943F0F1
:108A60004003A381F8BD3E60D5E700BF38B50C4692
:108A7000054608B1836BA3B1B4F90C00B8B1636EBD
:108A8000DB0701D4810515D528462146FFF75EFF97
:108A9000636EDA07054602D4A3899B050ED52846E6
:108AA00038BD00F017F8B4F90C000028E7D10546EE
:108AB000284638BDA06D00F037FAE5E7A06D00F05C
:108AC00035FA284638BD00BF014900F001BA00BFA1
:108AD00011AF00082DE9F0478246394800F024FA2A
:108AE000DAF83840002C66D1DAF80450354ACAF872
:108AF0003C200323CAE9B843DFF8CC90DFF8CC80F0
:108B0000334F344E04230AF53B72CAF8E82221465B
:108B1000C5E90243C5E90044C5E904446C6608227E
:108B2000AC6105F15C00FCF7B9FFC5E90759C5E97F
:108B30000987EE6205F1580000F0F2F9DAF8085002
:108B4000254BEB602146C5E90044C5E904446C6649
:108B5000AC60AC61082205F15C00FCF79FFFC5E941
:108B60000759C5E90987EE6205F1580000F0D8F908
:108B7000DAF80C50194BEB602146C5E90044C5E911
:108B800004446C66AC60AC61082205F15C00FCF743
:108B900085FF05F15800C5E90759C5E90A76C5F80A
:108BA000248000F0BDF90123CAF838300448BDE83C
:108BB000F04700F0BBB9BDE8F047014800F0B6B996
:108BC000DC0A0024C98A0008E19D0008059E00080F
:108BD000459E0008659E0008090001001200020081
:108BE000014800F0A1B900BFD80A0024014800F0F4
:108BF0009DB900BFD80A002438B5084B084D5B1B4F
:108C00009C1007D0043B1D44013C55F8043998479B
:108C1000002CF9D1BDE8384002F0A0BFD4BF000855
:108C2000D0BF0008F8B5244F0C46064600F0D8FC2B
:108C3000BA685568C4F57E630F3325F003052B44ED
:108C400023F47F6323F00F03A3F58054B4F5805F12
:108C500007DB0021304601F0B1F8BB682B44984295
:108C600004D0304600F0C2FC0020F8BD614230461E
:108C700001F0A4F801300DD0104ABB682D1B45F05F
:108C800001055D60136830461B1B136000F0AEFCED
:108C90000120F8BD0021304601F090F8BA68831A2F
:108CA0000F2BDEDD43F001035360054B03491B68C6
:108CB000C01A0860D5E700BF44040024E00A00247D
:108CC0004C080024002961D0F8B50C46064600F097
:108CD00087FC54F8042C7B4FA4F1080522F0010115
:108CE00005EB010CB868DCF80430604523F00303A1
:108CF00000F08B80D207CCF8043032D454F8082C22
:108D0000AD1A1144AA6807F1080082426AD00CEB40
:108D10000304D4F804E0EC68D4601EF0010FA260F4
:108D200000F0978041F001036B60CCF80010B1F5C2
:108D3000007F35D27A68CB08480901210133814090
:108D40001143796007EBC30257F83310083AC5E9BD
:108D5000021247F83350CD603046BDE8F84000F0CD
:108D600045BC0CEB03025268D00710D4194407F13C
:108D70000800DCF80830834273D0DCF80C20DA609D
:108D8000936041F001036B606950D0E7704741F098
:108D90000103B1F5007F44F8043CCCF80010C9D3BE
:108DA000B1F5206F4FEA512348D28B0903F1390006
:108DB00003F13802C300F818FB580838984259D01C
:108DC0005A6822F003028A4202D99B689842F7D17E
:108DD000D868C5E902308560DD603046BDE8F840FE
:108DE00000F004BC0CEB03025268D20763D40B44BE
:108DF000DCE90212CA60916043F001026A60304609
:108E0000EB50BDE8F84000F0F1BB0B44D10707D4AC
:108E100054F8082CAD1A1344D5E90212CA609160C7
:108E200043F001026A60284ABD6012689A4293D8F2
:108E3000264B30461968FFF7F5FE8DE7142B0AD94B
:108E4000542B1FD80B0B03F16F0003F16E02C3000C
:108E5000B1E719448DE703F15C0003F15B02C30045
:108E6000A9E741F00103C7E90455C5E902006B60B9
:108E7000695071E779689210012404FA02F20A43FA
:108E80007A60A6E7B3F5AA7F06D8CB0B03F178008A
:108E900003F17702C3008EE740F25452934206D8A2
:108EA0008B0C03F17D0003F17C02C30083E74FF4D8
:108EB0007E737E227FE741F001036B60CCF80010E7
:108EC0004AE700BF4404002450080024100B00248B
:108ED0002DE9F8430746884600F538764FF000093B
:108EE000D6E90154013D11D4A389012B05F1FF35C9
:108EF00008D9B4F90E300133214603D03846C047B3
:108F000049EA00096B1C04F16804EDD13668002EB3
:108F1000E6D14846BDE8F88300487047440900247C
:108F2000704700BF704700BF704700BF704700BF69
:108F30002DE9F0418B890C46990796B008D504F1CC
:108F400043030122C4E90432236016B0BDE8F08176
:108F5000B4F90E100029064627DB6A4602F0DAF85B
:108F6000002821DB019D05F47045A5F50055B5FAF3
:108F700085F54FF480686D094FF40067414630462F
:108F800000F07EF8B4F90C30F0B1204AF26343F0FF
:108F90008003C4F81480A3812060206135BB3B436B
:108FA000A38116B0BDE8F081A38913F0800519D024
:108FB0004FF040084146304600F062F80025B4F911
:108FC0000C302F460028E0D19A05BED423F00303CD
:108FD00004F1430243F002030121C4E90421A38107
:108FE0002260B2E74FF480682F46C7E7B4F90E104D
:108FF000304602F019FA10B9B4F90C30CFE7A38962
:1090000023F0030343F001031BB2C8E7C98A000839
:1090100070B50C46B1F90E10002996B015461E46E3
:1090200014DB6A4602F076F800280FDB019A02F49E
:109030007042A2F50052B2FA82F24FF480635209F4
:109040004FF4006032602B6016B070BDB4F90C10A4
:10905000002311F08000336004D0402218462A60BB
:1090600016B070BD4FF480632B6016B070BD00BFAA
:10907000024B0146186800F003B800BF100000243E
:109080002DE9F04F01F10B06162E83B0044624D8CB
:10909000102900F2BA8000F0A3FA1026182202204C
:1090A000B54F3A44A2F1080153688B4200F0BA80F0
:1090B0005A68D96822F003021A449D68E9608D60FD
:1090C000516841F001012046516003F1080500F0AC
:1090D0008DFA284603B0BDE8F08F36F0070600F1A0
:1090E0009480B14200F2918000F07AFAB6F5FC7FEC
:1090F000C0F09A81730A00F08F80042B00F26F8118
:10910000B30903F1390003F1380CC3009A4F3B4413
:10911000A3F108055B689D4206D10CE0002980F2AE
:109120002781DB689D4206D05A6822F00302911B1A
:109130000F29F3DD60463D69DFF840C265457CD00C
:109140006A6822F00302931B0F2B00F37B81002B34
:10915000C7E904CC80F26C81B2F5007F80F01A81FF
:10916000D308796801334FEA521E012202FA0EF247
:109170000A4357F833E0C5F808E007EBC3010839A4
:10918000E9607A6047F83350CEF80C508310012123
:109190009940914257D8114206D120F0030049006E
:1091A000114200F10400FAD007EBC0094D46864693
:1091B000D5F80C80454508D11DE1002B80F22481B3
:1091C000D8F80C80454500F01681D8F8042022F02C
:1091D0000302931B0F2BF0DD2046D8E9025408EB65
:1091E000060146F00106C8F80460EC60A56043F093
:1091F0000104C7E90411C1E902CC4C6048F802300F
:1092000000F0F4F908F1080502E00C2323600025C2
:10921000284603B0BDE8F08F4FF4007340204FF0B4
:109220003F0C73E7D3689A4208BF02307FF440AF27
:109230003D69DFF848C1654582D17A688310012114
:1092400099409142A7D9BD686B6823F003094E4548
:1092500003D8A9EB06030F2B7ADCDFF824B1494BC6
:10926000DBF800201B680132334405EB090A00F0EB
:10927000338103F580530F3323F47F6828F00F0800
:109280004146204600F09AFD411C024600F0F38062
:10929000824500F2EE803C4B196841441960084653
:1092A00000F04E81DBF80010019301311BBFA2EBEF
:1092B0000A0A5044CBF80020186012F0070B00F0A7
:1092C0001781CBF108010A44CBF580519044083155
:1092D000A1EB0801C1F30B0A51462046009200F0B1
:1092E0006DFD421CDDE9002300F04F81801A00EB88
:1092F0000A081968BA6048F001005144BD42506044
:10930000196000F02981B9F10F0F40F227816868D8
:10931000A9F10C0C2CF0070C00F0010040EA0C0045
:1093200068604FF0050E05EB0C00BCF10F0FC0E9B3
:1093300001EE00F2328150681546144B1A688A42D9
:1093400038BF1960124B1A688A4238BF196094E01E
:10935000AA1943F0010346F001066E602046BA6088
:10936000536000F043F90835284603B0BDE8F08F9C
:10937000D9681A44A1E600BF440400244C04002428
:109380004C080024100B0024E00A0024080B0024E1
:109390000C0B0024B2F5206F4FEA522363D3142B39
:1093A00000F2B78003F15C01C9005B3307EB010EEB
:1093B0007958AEF1080E8E4500F091804B6823F08D
:1093C0000303934202D989688E45F7D1D1F80CE0A6
:1093D0007A68C5E9021ECEF80850CD60D6E6142B97
:1093E00059D9542B00F29D80330B03F16F0003F128
:1093F0006E0CC3008AE60EF1010E1EF0030F05F19C
:1094000008057FF4D5AE51E0424445465368D8F88C
:109410000C1043F00103536055F8083F2046D96013
:109420008B6000F0E3F8F3E6F00806F1080237E697
:109430002A442046536843F001035360083500F086
:10944000D5F8E5E6A919204646F0010643F00104E7
:109450006E60C7E90411C1E902CC4C60AB5000F06A
:10946000C5F80835D4E6930903F13901C90038334A
:109470009CE7BD425FD0BD68686820F003084645A0
:10948000A8EB060302D80F2B3FF762AF204600F08F
:10949000ADF80025BCE603F15C0003F15B0CC300F2
:1094A00034E659F808394B4540F0968010F0030F28
:1094B00000F1FF30F5D17B6823EA01037B604900AE
:1094C00099423FF6C0AE19B9BDE649000EF1040E4F
:1094D0001942FAD0704667E603F11008D0E69A10F8
:1094E0004FF001087B6808FA02F21A437A6070E7CD
:1094F00002EB08014942C1F30B0A51462046009293
:1095000000F05CFC431CDDE900237FF4EFAEDA469B
:10951000EFE6542B25D8130B03F16F01C9006E330E
:1095200044E7B3F5AA7F25D8F30B03F1780003F1E4
:10953000770CC300EAE5294B186840441860B1E68F
:10954000CAF30B0CBCF1000F7FF4ACAEBD68C8448D
:1095500048F001006860F0E61546EEE6012353602E
:1095600094E7B3F5AA7F23D8D30B03F17801C900A0
:1095700077331BE740F25452934223D8B30C03F1E4
:109580007D0003F17C0CC300C0E5ABF1080BD844AF
:10959000A8EB02084FF0000AABE605F108012046EF
:1095A0000093FFF78FFBBD68009B68681968C4E6ED
:1095B00040F254518B420BD8930C03F17D01C9004A
:1095C0007C33F3E64FF47E737F204FF07E0C9DE5F5
:1095D0004FF47E717E23E9E67B6870E7E00A0024A1
:1095E0000148FFF7A1BC00BFD40A00240148FFF7DF
:1095F0009DBC00BFD40A0024C36C70B505460C4660
:109600004BB153F8240080B1026843F824200023B2
:10961000C0E9033370BD2122042101F02BFC034675
:10962000E8640028EDD1002070BD012101FA04F6A4
:10963000721D9200284601F01DFC0028F3D0C0E9FD
:109640000146E4E731B1C36C4A6853F82200086070
:1096500043F82210704700BF2DE9F0410D6907461D
:109660000E461C4601F1140E0020DEF800108BB2ED
:1096700002FB03434FEA134C090C02FB01CC0130FF
:109680009BB203EB0C4385424EF8043B4FEA1C446B
:10969000EBDC3CB1B368AB4207DD06EB850301357B
:1096A0005C6135613046BDE8F08171683846013152
:1096B000FFF7A2FF8046A8B13269023206F10C0121
:1096C00092000C30F7F76CFAFB6C726853F82210BA
:1096D000316043F82260464606EB850301355C6144
:1096E0003561DFE7024B03484246B52101F0A2FB9A
:1096F0003CBC0008D0BC0008020C12040346CAB9E6
:109700000304102013F07F4F04BF1B02083013F036
:10971000704F04BF1B01043013F0404F04BF9B0087
:109720000230002B05DB13F0804F00F1010008BF71
:10973000202070470020E5E70368024613F0070089
:1097400007D0D9071DD498071FD55B0813600120E7
:10975000704799B209B91B0C1020D9B209B9083069
:109760001B0A190704BF1B090430990704BF9B0893
:109770000230D90703D45B0800F1010003D0136065
:10978000704700207047202070479B08136002201C
:10979000704700BF38B5C36C04460D464BB15868DE
:1097A000B0B102685A6000220123C0E90435C260EA
:1097B00038BD2122042101F05DFB0346E06400284E
:1097C000EDD1094B094800224FF4A07101F032FBA2
:1097D0001C220121204601F04DFB0028F1D001227E
:1097E0000223C0E90123DEE73CBC0008D0BC00082E
:1097F0002DE9F04F0E691569AE4285B088461446D2
:1098000005DB2A46234635460C4616469846A3688D
:109810006168AF19BB42B8BF0131FFF7EDFE01909F
:10982000002800F08780019B03F1140909EB870AE7
:10983000D14505D24B46002243F8042B9A45FBD86C
:1098400008F1140808EB860B04F11403D8451A46F6
:1098500003EB85055FD22B1B153B23F00303043379
:109860001534A54238BF0423CDE902A7AC461F46F4
:10987000924605E0000C29D1C34509F1040948D9F5
:1098800058F8040B85B2002DF4D056464C46002300
:1098900056F8040B216882B21FFA81FE05FB02EE26
:1098A000000C0A0C734405FB002202EB13429BB22E
:1098B00043EA0243B44544F8043B4FEA1243E7D875
:1098C00049F8073058F8040C000CD5D0D9F800300E
:1098D000544619464D4600222688090C00FB061105
:1098E0000A449BB243EA024345F8043B54F8046B34
:1098F0002968360C8BB200FB063303EB1243A445F8
:109900004FEA1342E8D8C34549F8073009F1040982
:10991000B6D8DDE902A7002F02DC05E0013F03D045
:109920005AF8043D002BF9D0019B18461F6105B081
:10993000BDE8F08F034B0448019A40F25D1101F03D
:1099400079FA00BF3CBC0008D0BC000812F0030349
:109950002DE9F0411446064632D10D46A41020D020
:10996000D6F84880B8F1000F33D0E3074FF0000776
:1099700007D4641015D0D8F80000A8B18046E307DA
:10998000F7D5424629463046FFF732FFB5B1696840
:10999000F36C641053F821202A6043F821500546E7
:1099A000E9D12846BDE8F081424641463046FFF7FE
:1099B0001FFFC8F8000007608046E0E70546D8E7CB
:1099C000013B0F4A52F823200023FFF745FE0546CE
:1099D000C4E701213046FFF70FFE804640B1012366
:1099E00040F27122C0E904320023B0640360BCE796
:1099F000044B054842464FF4A07101F01BFA00BF2A
:109A000040BE00083CBC0008D0BC00082DE9F0476F
:109A10000C4690462669A368496806EB6216751CD9
:109A20009D4207464FEA621904DD5B009D4201F149
:109A30000101FADC3846FFF7DFFD8446002851D0EB
:109A4000B9F1000F00F114000EDD09F105024FEA33
:109A5000820E03460CEB8202002143F8041B934262
:109A6000FBD1AEF114031844216904F1140318F07A
:109A70001F0803EB81012DD0C8F1200986464FF065
:109A8000000A1A6802FA08F242EA0A024EF8042BA7
:109A900053F8042B994222FA09FAF2D80B1B153B12
:109AA00023F00303043304F11502914238BF042369
:109AB000BAF1000F18BF2E4640F803A0FB6C626895
:109AC000CCF8106053F822102160604643F8224021
:109AD000BDE8F087043853F8042B40F8042F99426E
:109AE000F9D8EBE7034B0448624640F2D91101F084
:109AF000A1F900BF3CBC0008D0BC00080B6984463B
:109B00000069C01A15D10CF1140C14310CEB83024E
:109B100010B401EB830301E0944508D252F8044DE0
:109B200053F8041D8C42F7D004D24FF0FF3010BC24
:109B300070477047012010BC704700BF2DE9F84FF7
:109B40000F691369FF1A002F0E4690467AD101F172
:109B50001405143202EB830205EB830301E09D42FE
:109B600073D253F8041D52F8044DA142F7D064D3C8
:109B70007168FFF741FD8146002872D03569D8F839
:109B80001020C76008F1140E06F1140009F1140A40
:109B900006F1100C0EEB820200EB85075646002101
:109BA0005EF8044B5CF804BFA3B211FA8BF1CB1A38
:109BB000210CC1EB1B4101EB23419BB243EA014362
:109BC000724546F8043B4FEA2141E9D8A2EB08046C
:109BD000153C08F11508424524F0030606F1040679
:109BE00038BF0426304424F0030238BF00228742E5
:109BF0005244B24416D95646044654F8043B11FA6E
:109C000083F10A1402EB134289B241EA0243A742EC
:109C100046F8043B4FEA2241EFD87A1E101A20F092
:109C20000302524423B952F8043D013D002BFAD0FF
:109C3000C9F810504846BDE8F88F3346012746461C
:109C4000984695E7F9DB002792E70021FFF7D4FC5F
:109C5000814668B101220023C9E904234846BDE8D2
:109C6000F88F074B07484A464FF4107101F0E2F8AD
:109C7000034B04484A4640F2322101F0DBF800BFB2
:109C80003CBC0008D0BC000870B5012182B016466B
:109C90001D46FFF7B1FC044600284BD02B46C5F308
:109CA0000A55C3F313030DB143F48013002E01933F
:109CB00022D068460096FFF73FFD002836D0019B72
:109CC0000099C0F1200203FA02F20A43C340019353
:109CD0006261002B14BF02210121A3612161ADB19A
:109CE000069AA5F2334303441360079BC0F1350085
:109CF0001860204602B070BD01A8FFF71DFD019B52
:109D00000121C4E904132030002DE9D104EB8102C4
:109D1000A0F232431069069A1360FFF7EDFC079B2F
:109D2000C0EB41112046196002B070BDDDE900238F
:109D30006261CEE7034B0448224640F20A3101F04B
:109D400079F800BF3CBC0008D0BC0008DFF860C058
:109D5000F8B521F000430027634504460D4616463A
:109D6000176022DC844653EA0C0C1ED0DFF844C096
:109D700001EA0C0C0A46BCF1000F09D10E4B00227F
:109D8000F7F7E8F96FF0350704460A4621F000437B
:109D900022F0FF421B1522F4E002A3F2FE3342F050
:109DA0007F553B4445F40015336020462946F8BDF5
:109DB000FFFFEF7F0000F07F0000504338B5074DF4
:109DC0000022044608462A60F7F79EFE431C00D096
:109DD00038BD2B68002BFBD0236038BD140B00244A
:109DE00010B50C46B1F90E1001F0DEFB002803DBC4
:109DF000236D0344236510BDA38923F48053A381FD
:109E000010BD00BF2DE9F0410C46B1F90C101F4602
:109E1000CB05054616460BD421F48051A1813B4663
:109E2000B4F90E1032462846BDE8F04100F0A6BF56
:109E3000B4F90E100223002201F00EFBB4F90C104D
:109E4000EAE700BF10B50C46B1F90E1001F004FBB3
:109E5000A389421C0EBF23F4805343F48053206532
:109E6000A38110BDB1F90E1001F040B830B540EA41
:109E70000104A30701D1032A0FD8844601F1FF3E54
:109E800007E01EF8011F03F8011B541EC1B19C46D8
:109E900022466346002AF4D130BD0B46844619465B
:109EA00053F8045BA5F1013424EA050414F0803F63
:109EB000E4D1043A032A4CF8045B1946EFD8DDE7F5
:109EC0006244002CE8D003F8011B9342FBD130BD63
:109ED0002DE9F84F4B6E9C0490462DD5936812687F
:109EE00043B38B46064602F1080959E9025A5FEA74
:109EF0009A0715D0043D002401E0A7420ED055F882
:109F0000041F5A46304601F0D1F8431C04F1010405
:109F1000F3D10023C8E90133BDE8F88FD8F8083041
:109F20002AF0030AA3EB0A03C8F8083009F108096C
:109F3000002BDAD10020ECE701F002F90023C8E998
:109F40000133BDE8F88F00BF10B4946814B110BCA1
:109F5000FFF7BEBF2046546010BC70472DE9F04F9C
:109F6000BDB0CDE904301C460191174618B1836B92
:109F7000002B00F08682019A536EDE0740F18F813C
:109F8000B2F90C108AB2900408D441F4005201993D
:109F90004B6E8A8123F4005392B24B66110740F155
:109FA000F780019B1B69002B00F0F28002F01A037E
:109FB0000A2B00F0FB8013AB10930023CDE9113383
:109FC000CDE90A3308930DF14C09099303933B78CB
:109FD000002B00F051813C4604E014F8013F002BB7
:109FE00000F02C81252BF8D1E51B40F02981237846
:109FF000002B00F041814FF0000300258DF83B302D
:10A00000671C637802954FF0FF3B2B240137A3F1C7
:10A0100020025A2A00F25281DFE812F09802500121
:10A02000500194025001500150016A00500150014A
:10A0300036026B0250014102A6025001A2025B00EF
:10A040005B005B005B005B005B005B005B005B0038
:10A050005001500150015001500150015001500178
:10A060005001230284005001500150015001500161
:10A0700050015001500150015001DD0050015001CC
:10A080005001070250015902500150011E055001B4
:10A090005001500150015001500150015001500138
:10A0A0005001230286005001500150014F028600EA
:10A0B00080005001450250018102DF006F028000E4
:10A0C000500107027E003E0550015001400550013D
:10A0D0007E00A3F13002002117F8013B01EB810162
:10A0E00002EB4101A3F13002092AF5D902918EE772
:10A0F000DDF814804046FEF70FFF43680A931846C8
:10A10000F6F7FEFD0B9006464046FEF705FF836816
:10A110000993002E40F07B843B7877E73B7845F04D
:10A12000200573E745F01005AC06049E40F16F81F1
:10A13000073626F007063246736852F8086B049219
:10A140009846002BC0F22D84BBF1FF3F00F0108534
:10A1500056EA080325F0800A00F008840A2E78F1F8
:10A16000000380F0BD84303601238DF8EF60554642
:10A1700000930DF1EF04DDF800809DF83B30D845E9
:10A18000B8BFD846002B00F0A88008F10108A4E071
:10A19000019D05982946FDF769FB002840F0888558
:10A1A000AA8902F01A030A2B7FF405AF0199B1F9CD
:10A1B0000E30002BFFF6FFAE4B6EDE0702D4950586
:10A1C00040F156850199059823463A463DB0BDE8D1
:10A1D000F04F00F093BD45F0100515F0200800F099
:10A1E0000781049E073626F007063346D6F804801A
:10A1F00053F8086B049325F4806A00234FF00002A3
:10A200008DF83B20BBF1FF3F00F0C88156EA080201
:10A210002AF0800540F0C181BBF1000F40F0AB8413
:10A22000002B40F0A8831AF00103009300F0D683BE
:10A2300030238DF8EF300DF1EF049CE7E51B1BD0C8
:10A24000119B129A01332A44072BC9E90075129217
:10A25000119305DC09F10809039B2B440393C6E61F
:10A26000002A00F07F830199059810AAFFF730FEBD
:10A2700040B90DF14C09EFE7129B002B40F0098526
:10A2800000231193019A536ED90740F1A680938958
:10A290005B0600F1198503983DB0BDE8F08F019B86
:10A2A000B3F90C108D058AB23FF56DAE1D46986D61
:10A2B000FEF73AFEB5F90C108AB264E6002BDBD04B
:10A2C0008DF88C304FF001084FF000038DF83B30D3
:10A2D000CDF8008023AC4FF0000B15F0020306937D
:10A2E00018BF08F1020815F08403079305D1029BFB
:10A2F000A3EB0806002E00F36C82DDE91121501C4F
:10A300009DF83B608EB10DF13B020131C9F8002090
:10A3100007284FF00102CDE91101C9F8042000F32C
:10A320003B82024609F108090130069BDBB10FAB05
:10A330000231C9F8003007284FF00203CDE91101BE
:10A34000C9F8043040F34082002900F006830199E7
:10A35000059810AAFFF7BCFD002893D1DDE9112173
:10A360000DF14C09501C079B802B00F05881009B7D
:10A37000ABEB0306002E00F3B681009BC9F800404A
:10A3800019440728CDE91101C9F8043040F344818C
:10A39000002900F072820199059810AAFFF798FD34
:10A3A00000287FF46FAF12990DF14C09680705D5AD
:10A3B000029BA3EB0804002C00F36982DDE9022371
:10A3C0004245ACBF9B1843440393002940F0D5811C
:10A3D000002311930DF14C09F9E5019B9B899A0526
:10A3E0003FF556AF019CA06DFEF7A0FDA3894FE796
:10A3F00015F0100340F0238315F0400200F0EB83CA
:10A40000049A52F8046B04929846B6B2F3E656F8F2
:10A41000043B0496E80600F1ED82690640F1E7820C
:10A4200043F3C0381EB243468BE6049E56F8044BF5
:10A430004FF000038DF83B30002C00F0B183BBF1EE
:10A44000FF3F00F02E835A4600212046F6F758FBC6
:10A45000002800F01284031B009304964FF0000BB9
:10A4600089E6049E4FF000038DF83B304FF0010861
:10A4700056F8043B8DF88C300496CDF8008023AC60
:10A4800029E7FEF727FB76E5049B53F8042B02929D
:10A49000002A80F29F82029A0493524202923B78F1
:10A4A00045F00405B2E53B786C2B03BF7B7845F0A3
:10A4B0002005013745F01005A8E53B78682B03BF60
:10A4C0007B7845F40075013745F040059EE545F081
:10A4D000100A1AF0200800F05582049E073626F074
:10A4E00007063346D6F8048053F8086B049301231B
:10A4F00084E63B788DF83B4088E5049B53F8046B79
:10A50000049330238DF83C3078238DF83D30B94BDF
:10A51000089345F0020A4FF0000802236EE6AE06EB
:10A5200000F18382EC0600F13383680600F1928328
:10A53000A90540F12D83049E039A56F8043B049626
:10A540001A7044E53B7845F001055FE59DF83B3026
:10A55000002B7FF4E1AD20238DF83B303B7855E5AF
:10A560003B7845F0800551E5394611F8013B2A2B2F
:10A5700000F0B383A3F13002092A0F464FF0000B1D
:10A580003FF645AD17F8013B0BEB8B0B02EB4B0B8A
:10A59000A3F13002092AF5D939E5AA46012B3FF487
:10A5A000DDAD022B3CAC12D1089A06F00F03360940
:10A5B000D35C04F8013D46EA08764FEA181856EADB
:10A5C0000803F2D13CAB1B1B55460093D3E506F0C4
:10A5D0000703F60846EA48764FEAD808303356EAC9
:10A5E0000801224604F8013DF1D11AF0010FE9D02B
:10A5F000302BE7D03023023A04F8013C3CAB9B1AE5
:10A60000554600931446B6E500991394012314911E
:10A61000129111930DF14C0909F10809C6E6029B4C
:10A62000A3EB0806002E7FF7A2AE102E40F3518355
:10A63000DFF8C4A15346CDE906B4BA46DDF814B03C
:10A64000019C2F461D4607E002F1020C09F10809A2
:10A650000246103E102E1EDD501C1031102307281C
:10A66000CDE91101C9F80050C9F80430ECDD10AA99
:10A67000002900F08B80214658460DF14C09FFF768
:10A6800027FC00287FF4FEADDDE91121103E102EDD
:10A6900002F1010CE0DCDDE906B42B463D465746ED
:10A6A0009A463144BCF1070FCDE911C1C9F800A0A9
:10A6B000C9F8046040F39581002900F0BB8201993C
:10A6C000059810AAFFF704FC00287FF4DBAD009B7F
:10A6D000DDE91121ABEB0306002E02F101000DF1C3
:10A6E0004C097FF74AAE102EDFF80CA131DD53463E
:10A6F000CDE90645BA46059C019D4FF0100B1F465B
:10A7000007E002F1020C09F108090246103E102E82
:10A7100019DD501C10310728C9E9007BCDE9110172
:10A72000EFDD10AA19B3294620460DF14C09FFF7B9
:10A73000CFFB00287FF4A6ADDDE91121103E102EDD
:10A7400002F1010CE5DCDDE906453B466046574673
:10A750009A4631440728CDE91101C9F800A0C9F88B
:10A76000046000F3E68009F10809013005E64FF0C6
:10A77000010C0A460DF14C09C8E70199059810AA89
:10A78000FFF7A6FB00283FF423AE7BE54FF0010C5A
:10A790000A460DF14C095CE7002900F0DB800199C5
:10A7A000059810AAFFF794FB00287FF46BADDDE954
:10A7B00011210DF14C09501CB7E502210FAB14918A
:10A7C000139301200DF14C09024609F10809501CB0
:10A7D000C9E5102E40F35782DDE911C1DFF81CA056
:10A7E000CDE90CB410235446DDF804B0DDF814A014
:10A7F00062460DE0D8BB00085CBE00084CBE0008F5
:10A8000002F1020C09F108090246103E102E1BDD70
:10A81000501C10310728C9E90043CDE91101EFDDD3
:10A8200010AA21B3594650460DF14C09FFF750FBD1
:10A8300000287FF427ADDDE91121103E102E02F132
:10A84000010C4FF01003E3DCA246DDF830B00D9CA4
:10A8500062463144072ACDE91121C9F800A0C9F8A0
:10A86000046000F3A78009F10809501C48E50A4676
:10A870004FF0010C0DF14C09C7E76C07119150D551
:10A88000029BA3EB0804002C4BDD0DF14C09102CAE
:10A8900040F30982DFF8ECA2119A059EDDF804B0BE
:10A8A00053461025BA461F4606E0901C09F10809D8
:10A8B0001A46103C102C19DD531C1031072BC9E926
:10A8C0000075CDE91131F0DD10AA29B359463046A3
:10A8D000FFF7FEFA00287FF4D5ACDDE91121103C2A
:10A8E000102C02F101000DF14C09E5DC3B46574606
:10A8F0009A4621440728C9E900A4CDE911017FF750
:10A900005DAD71B10199059810AAFFF7E1FA002831
:10A910007FF4B8AC129951E501200A460DF14C09BB
:10A92000C7E7DDE902234245ACBF9B1843440393CC
:10A930004EE500293FF468AE0199059810AAFFF78B
:10A94000C7FA00287FF49EAC1198129901300DF1DE
:10A950004C0912E5069B002B77D101200A460DF128
:10A960004C0900E511920DF14C0975E4BBF1000FA3
:10A970007FF4F9AB55464FF0000BCDF800B03CAC7E
:10A98000FFF7F9BB1AF010033AD11AF0400200F0B9
:10A990001381049A52F8046B04929846B6B20123CC
:10A9A0002CE42D2376428DF83B3068EB4808AA460C
:10A9B000012327E400297DD00199059810AAFFF70B
:10A9C00087FA00287FF45EACDDE911210DF14C0916
:10A9D000501C95E404933B78FFF718BB3CACFFF7A1
:10A9E000CABB09F108090CF101006246BFE4AA05DF
:10A9F00000F138814FEAE3781E464346FFF7A1BBDA
:10AA0000049B53F8046B04930123FFF7F7BB099BE6
:10AA1000002B3FF481AB099B1B78002B3FF47CABF0
:10AA20003B7845F48065FFF7F1BADDE9031656F887
:10AA3000042B0496CB17C2E90013FFF7C8BA049B96
:10AA400053F8046B0493FFF7D6BB02210FAB1491AC
:10AA500013930DF14C09B8E64B4A089215F0200803
:10AA600036D0049E073626F007063246D6F8048014
:10AA700052F8086B0492EA0709D556EA080206D094
:10AA80008DF83D30302345F002058DF83C3025F43B
:10AA9000806A0223FFF7B2BBAA461AE53B4A089236
:10AAA000DCE720460496F6F72BF94FF0000B0090F8
:10AAB000FFF761BB9DF83B20002A00F0C180012018
:10AAC0000DF13B02149013920DF14C09014628E45C
:10AAD00015F0100242D0049A52F8046B0492CAE7AF
:10AAE0000AF48063CDF800B0CDF81890BB46DDF8CD
:10AAF000249000253CAC1F4609E030464146F5F75E
:10AB00007DFE0A2E78F100031BD3064688463046A8
:10AB100041460A220023F5F771FE1146303104F850
:10AB2000011C0A220023013C0135002FE5D099F8D1
:10AB30000010A942E1D1FF2DDFD00A2E78F10003E9
:10AB400064D23CAB1B1BCDF824905F46DDF8189017
:10AB5000DDF800B000935546FFF70DBB15F040013E
:10AB600047D0049951F8046B04919046B6B282E73D
:10AB7000AA46FFF7F3BA012BAA467FF412ADFFF7FE
:10AB8000F2BA00BF4CBE0008ECBB0008D8BB0008FE
:10AB9000049E039A56F8043B1A600496FFF717BA0E
:10ABA000BBF1060FD84628BF4FF00608504CCDF831
:10ABB00000800496FFF78FBB049B1AF4007814BF43
:10ABC00053F8046B53F8046B04931CBF9046F6B221
:10ABD0000123FFF713BB049B15F4007814BF53F84F
:10ABE000046B53F8046B04931CBF9046F6B2FFF756
:10ABF00002BB049A15F4007814BF52F8046B52F8A3
:10AC0000046B04921CBF8846F6B234E70B9B0A998A
:10AC1000E41A1A462046FFF729F999F801300BB1DA
:10AC200009F10109304641460A2200230025F5F7C3
:10AC3000E5FD6AE701200A460DF14C09FFF797BBD5
:10AC4000069B002B7FF4B9AD0A4601200DF14C099B
:10AC5000FFF78DBB049E039A56F8043B04961A80B6
:10AC6000FFF7B5B943F3C0185EB24346FFF769BAC0
:10AC7000886DFEF75BF9FFF7A5BACDF800B0049632
:10AC80008346FFF778BA119A1299DFF868A001326B
:10AC9000DFE50199059810AAFFF71AF900283FF49B
:10ACA000EFAAFFF7EFBA1198DFF848A0013020E6CD
:10ACB000019B5B6EDB0707D4019B9B899F0503D437
:10ACC000019B986DFEF732F94FF0FF330393FFF7C6
:10ACD000E2BADFF824A08446E3E4049A7B780F46C6
:10ACE00052F8041B049241EAE17BFFF78FB900BFE1
:10ACF00000BC00084CBE00085CBE0008F0B51F4652
:10AD00008B89ADF26C4D23F00203ADF80C304B6E25
:10AD10001993CB89ADF80E30CB6907934B6A099331
:10AD20001AAB009304934FF48063154606460293D2
:10AD3000059316A800230C460693FEF7F1F82A4661
:10AD40003B4669463046FFF709F9051E07DB6946B1
:10AD50003046FDF78BFE002818BF4FF0FF35BDF8D9
:10AD60000C305B0603D5A38943F04003A3811698FA
:10AD7000FEF7D8F828460DF26C4DF0BD38B50C46FC
:10AD8000084D8446114620461A4600232B6064462F
:10AD9000F6F716FE431C00D038BD2B68002BFBD005
:10ADA000236038BD140B00242DE9F047DFF87CA0A8
:10ADB0000646DAF8000098460F469146FEF7B4F8CA
:10ADC0001B4B1B68D3F8484124B365681F2D26DC54
:10ADD0005EB96B1C0235DAF80000636044F8257038
:10ADE000FEF7A4F80020BDE8F08704EB85010123FD
:10ADF000C1F88890D4F88821AB401A43022EC4F8D9
:10AE00008821C1F80881E4D1D4F88C211343C4F817
:10AE10008C31DEE703F5A674C3F84841D5E7DAF8CC
:10AE20000000FEF783F84FF0FF30DCE74004002419
:10AE3000C4BB000800B50B4C25681446EE681A46E2
:10AE400085B003460D464CB107490095CDE9011484
:10AE50003046064900F0C2F800F02CFE04490C46CA
:10AE6000F3E700BF100000246CBE00087CBE0008A1
:10AE700074BB000838B5A1FB02148CBBFEF700F9C7
:10AE80000546E0B150F8042C22F00302043A242ACB
:10AE900017D8132A1AD91B2AC0E900441DD9242A1D
:10AEA00014BF00F1100200F118024FF00003C0E9D6
:10AEB000024404BF04614461C2E900339360284640
:10AEC00038BD2146FAF7EAFD284638BD0246002380
:10AED000C2E900339360284638BD00F10802F6E766
:10AEE000FAF7B2FD0C2300250360E8E738B5074DFB
:10AEF0000022044608462A60F6F77CFD431C00D079
:10AF000038BD2B68002BFBD0236038BD140B002408
:10AF100070B500294BD006460C4610B1836B002B50
:10AF200048D0636ED80734D5B4F90C30002B3ED02E
:10AF300021463046FDF70AFDE36A054633B1E16973
:10AF4000304698470028B8BF4FF0FF35A3891A064E
:10AF50003BD4216B41B104F14003994202D0304609
:10AF6000FDF7B0FE00232363616C21B13046FDF78D
:10AF7000A9FE00236364FDF733FE636E0022DB0746
:10AF8000A28127D5A06DFDF7CDFFFDF72FFE284646
:10AF900070BDA3899905CBD4A06DFDF7C5FFB4F9A9
:10AFA0000C30002BC4D1656E15F0010508D00025CA
:10AFB000284670BDFDF78EFD636ED807B4D4E8E770
:10AFC000A06DFDF7B3FF284670BD21693046FDF73F
:10AFD00079FEBEE7A06DFDF7A9FFD3E70EB410B56B
:10AFE00083B005AB064C53F8042B0193014620684F
:10AFF000FEF7B4FF03B0BDE8104003B0704700BFD8
:10B00000100000242DE9F04383B00746884614461B
:10B0100000F01CFA012803D108F1FF33FE2B37D9C9
:10B02000424604F15C0301A9384600F017FD421CBA
:10B03000064633D038B39DF804C00DF1050900254C
:10B0400009E023685A1C226083F800C00135B5422C
:10B0500019D219F801CBA368013B002BA360F0DAE9
:10B06000D4F818E0734561462246384602DBBCF14D
:10B070000A0FE6D100F09AFC431CE7D106463046A1
:10B0800003B0BDE8F0834646304603B0BDE8F08328
:10B090005FFA88FC8DF804C00646CEE7A3893046E7
:10B0A00043F04003A38103B0BDE8F08330B5536E95
:10B0B00013F0010FB2F90C30144683B005469AB272
:10B0C00001D198051CD5900406D4626E43F4005358
:10B0D00042F40052A381626622462846FFF792FF9F
:10B0E000636EDA07054602D4A3899B0502D528467C
:10B0F00003B030BDA06DFDF719FF284603B030BD89
:10B10000A06D0191FDF710FFB4F90C3001999AB2CE
:10B11000D9E700BF70B50C46084D0346002620460F
:10B1200011461C462E60F6F791FC431C00D070BD02
:10B130002B68002BFBD0236070BD00BF140B0024D4
:10B140009368002B00F081802DE9F04FB1F90C30AD
:10B150000C461907804683B0174698B223D5236959
:10B160000BB310F002033D682BD04FF0000ADFF85C
:10B17000B4B256465E453346524628BF5B4640460B
:10B18000002E4FD0E169D4F824C0E047002852DDFA
:10B19000BB681B1A8244361ABB60002BEAD1002020
:10B1A00003B0BDE8F08F21464046FCF75FFB002866
:10B1B00040F03481B4F90C303D6898B210F00203CD
:10B1C000D3D110F0010942D14E463EB38205D4F8E6
:10B1D00008B040F18180B3455A4600F2B18010F4C6
:10B1E000906F40F0BE8020680192494600F060F9FF
:10B1F000A3682168019AA3EB0B030A44B246A3603B
:10B2000022600026B868A0EB0A00D144B86000288C
:10B21000C5D0B4F90C0080B2002ED7D1D5E9009684
:10B220000835D2E7D5E900A60835A3E72146404610
:10B23000FDF71CFC80B3B4F90C3043F040034FF031
:10B24000FF30A38103B0BDE8F08F002070471E4699
:10B25000AA46994618461D4656B388B34A46D4E9CD
:10B2600004132068B24228BF3246884205D9A1683B
:10B2700003EB010B5A4500F3A780934264DCE169BC
:10B28000D4F824C02A464046E047B0F1000BD2DD96
:10B29000B9EB0B09CAD00120BB68A3EB0B035D44DB
:10B2A000A6EB0B06BB60002B3FF479AF002ED4D188
:10B2B0000AF1080353E902569A460833002EF9D0E2
:10B2C00032460A212846F5F71BFC002800F09D8035
:10B2D0000130A0EB0509C1E720682369984217D81F
:10B2E0006369B34214D86FF00042B24228BF3246BD
:10B2F000E16992FBF3F2D4F824C002FB03F3404669
:10B300004A46E047B0F1000A95DDA6EB0A0679E768
:10B31000B345DA4628BFB2465246494600F0C8F85F
:10B32000A3682268A3EB0A035244A3602260002BA7
:10B33000EBD121464046FDF799FB0028E5D07AE79E
:10B340002068B34632464FE72946019200F0B0F834
:10B35000019AA3689B1AA360236813442360934651
:10B3600096E723682169A3EB010B636903EB430AAA
:10B370000AEBDA7A0BF101034FEA6A0A33445345C8
:10B38000524684BF9A46524643052CD51146404644
:10B39000FDF776FE00283BD05A4621690190F5F76B
:10B3A000FFFBA289019B22F4906242F08002A281FD
:10B3B00003EB0B002361AAEB0B03C4F814A0A360FA
:10B3C0002060B34632460FE729465A4600F070F82F
:10B3D00023685B44236021464046FDF747FB002875
:10B3E0003FF456AF27E7404600F0F4F80346002844
:10B3F000DED121694046FDF765FCB4F90C300C2222
:10B4000023F08003C8F8002017E7721C914626E756
:10B410000C22B4F90C30C8F800200EE74FF0FF30D2
:10B42000BEE600BF00FCFF7F38B5074D0022044692
:10B4300008462A60F6F7B8FA431C00D038BD2B68DE
:10B44000002BFBD0236038BD140B0024014B93F874
:10B45000280170475408002438B50C46084D84462E
:10B46000114620461A4600232B606446F6F7CEFAB2
:10B47000431C00D038BD2B68002BFBD0236038BDA7
:10B48000140B002482B049B15AB16BB113780B6030
:10B490001278101E18BF012002B0704701A9002ABF
:10B4A000F3D1104602B070476FF00100F4E700BF1F
:10B4B00088420DD98B1883420AD900EB020CBAB12D
:10B4C000624613F801CD02F801CD9942F9D17047D7
:10B4D0000F2A0ED8034602F1FF3C4AB10CF1010CD1
:10B4E000013B8C4411F8012B03F8012F6145F9D180
:10B4F000704740EA01039B0750D1A2F1100370B5D9
:10B5000001F1200C23F00F0501F1100E00F11004E1
:10B51000AC441B095EF8105C44F8105C5EF80C5CEF
:10B5200044F80C5C5EF8085C44F8085C5EF8045C67
:10B5300044F8045C0EF1100EE64504F11004E9D164
:10B54000013312F00C0F01EB031102F00F0400EBBA
:10B55000031327D0043C24F003064FEA940C1E4446
:10B560001C1F8E465EF8045B44F8045FB442F9D1B8
:10B570000CF1010402F0030203EB840301EB8401EC
:10B5800002F1FF3C4AB10CF1010C013B8C4411F873
:10B59000012B03F8012F6145F9D170BD02F1FF3C89
:10B5A00003469BE72246EBE738B50C46084D844638
:10B5B000114620461A4600232B606446F6F72EFA01
:10B5C000431C00D038BD2B68002BFBD0236038BD56
:10B5D000140B00242DE9F84F1746002900F098803D
:10B5E00007F10B0580460C46FDF7FAFF162D5DD8D6
:10B5F00010252A46AF425ED854F8041C21F00306F9
:10B600009642A4F1080962DABC4BD3F808C009EBF2
:10B610000600844500F09780D0F804C02CF00103A8
:10B6200003445B68DB0768D42CF0030C06EB0C03C7
:10B63000934247DACB0710D454F8083CA9EB030A2D
:10B64000DAF8043023F003018C44B444944580F2CA
:10B6500011817318934280F2E88039464046FDF725
:10B660000FFD0746E0B154F8043C23F001034B44BE
:10B67000A0F10802934200F0D280321F242A00F287
:10B68000F580132A00F2AC80034622461168196047
:10B690005168596092689A6021464046FDF712FB56
:10B6A0004046FDF7A3FF3846BDE8F88F25F00705B3
:10B6B000002D2A469EDA0C23C8F8003000273846B1
:10B6C000BDE8F88F1E46D0E90223D3609A60731B51
:10B6D0000F2B22D8D9F8043003F0010333434E4432
:10B6E000C9F80430736843F001037360404627468D
:10B6F000FDF77CFF3846BDE8F88FC907ADD454F894
:10B70000083CA9EB030ADAF8041021F00301A0E7D2
:10B71000BDE8F84F1146FDF7B3BCD9F8041001F0AD
:10B7200001012943C9F8041009EB05014E4443F017
:10B7300001034B60736843F00103083173604046B6
:10B74000FDF7C0FAD2E7DCF8040020F0030B06EBAB
:10B750000B0C05F1100084454DDAC9073FF57DAFAC
:10B7600054F8081CA9EB010ADAF8041021F00301CF
:10B770008B44B34458453FF76CAF5746DAF80C108A
:10B7800057F8080F321F242AC160886000F2DB805E
:10B79000132A40F2D6802168CAF808106168CAF8F6
:10B7A0000C101B2A00F2DF8008340AF11002216815
:10B7B000116061685160A16891600AEB0501ABEB13
:10B7C000050242F0010299604A60DAF8043003F0A1
:10B7D00001031D434046CAF80450FDF707FF6EE71A
:10B7E00023680360636843601B2A68D804F1080279
:10B7F00000F108034AE709EB05029A60ACEB050388
:10B8000043F00103536054F8043C03F001031D436B
:10B81000404644F8045CFDF7E9FE27464FE750F840
:10B82000043C23F003031E4451E75746DAF80C109A
:10B8300057F8080F321F242AC16088604CD8132A99
:10B8400048D92168CAF808106168CAF80C101B2A88
:10B8500056D808340AF110021E4623681360636844
:10B860005360A3689360D1463C4630E72146FFF71A
:10B870001FFE11E7D0E902135746CB60996057F8D5
:10B88000081FDAF80C30CB60321F242A99602DD8BB
:10B89000132A29D92368CAF808306368CAF80C301B
:10B8A0001B2A42D808340AF1100322681A60626821
:10B8B0005A60A2689A606646D1463C4607E7A3688C
:10B8C0008360E368C360242A26D004F1100200F1EB
:10B8D0001003DBE63A46BFE7214638461E46D1460E
:10B8E000FFF7E6FD3C46F2E63B46DEE721463846FA
:10B8F0006646D146FFF7DCFD3C46E8E644040024FA
:10B90000A168CAF81010E168CAF81410242A20D0DF
:10B9100010340AF118029FE72369036161694161EC
:10B9200004F1180200F11803B0E6A368CAF8103059
:10B93000E368CAF81430242A21D010340AF118031D
:10B94000B3E73A4633E721463846FFF7B1FD164BD9
:10B9500033E72269CAF818206269CAF81C20183433
:10B960000AF1200278E7A168CAF81010E168CAF865
:10B970001410242A0DD010340AF1180217E7236995
:10B98000CAF818306369CAF81C3018340AF1200369
:10B990008BE72269CAF818206269CAF81C2018349B
:10B9A0000AF1200203E700BF44040024F8B50D4665
:10B9B0001446064610B1836B002B43D0B4F90C201B
:10B9C000A369A360170790B21BD52369CBB1EDB271
:10B9D00081042F4622D522686169D31A994229DD54
:10B9E0000133A1680139A160511C216015706269A1
:10B9F0009A422AD0A389DB0701D50A2D25D03846E3
:10BA0000F8BD21463046FBF731FF20BBB4F90C20CE
:10BA1000236990B2EDB281042F46DCD442F4005287
:10BA2000A281626E616922F4005262662268D31AB2
:10BA30009942D5DC21463046FDF718F858B92268FE
:10BA40000123CEE7FDF746F8B8E721463046FDF77B
:10BA50000DF80028D3D04FF0FF37D0E770B505467A
:10BA600084B01C4639B10B4ED6F8E060B047431C99
:10BA700009D004B070BD0A460649D1F8E06001A9BA
:10BA8000B047431CF5D100228A2322602B6004B00A
:10BA900070BD00BF5408002449B1FF2A02D80A70C3
:10BAA000012070478A2303604FF0FF30704708463B
:10BAB000704700BF08B5062000F004F80120F6F733
:10BAC0001DF800BF38B5154B1F281D6820D8D5F8C4
:10BAD000DC22044662B152F820304BB1012B15D064
:10BAE000591C0FD0002542F820509847284638BDF1
:10BAF000284600F02BF8224601462846BDE838408B
:10BB000000F00EB816232B60012038BD002038BD90
:10BB100016232B604FF0FF3038BD00BF100000240B
:10BB200070B50C46084D03460026204611461C46BB
:10BB30002E60F5F7DBFF431C00D070BD2B68002B97
:10BB4000FBD0236070BD00BF140B0024F5F7CCBF01
:10BB5000F8B500BFF8BC08BC9E467047F8B500BFFA
:08BB6000F8BC08BC9E467047CA
:10BB6800656E636F6465723A25640D0A0000000013
:10BB780073746172742074696D653A256C750D0A69
:10BB88000000000000000000010203040102030499
:10BB980006070809010002000400060008000A0060
:10BBA8000C0010002000400080000001080402047E
:10BBB8000801010101010103070100001800002428
:10BBC800494E4600696E66004E414E006E616E0039
:10BBD80030313233343536373839616263646566FB
:10BBE80000000000303132333435363738394142BD
:10BBF8004344454600000000286E756C6C2900001F
:10BC0800300000002020202020202020202020207C
:10BC1800202020203030303030303030303030305C
:10BC2800303030304E614E00496E66696E69747905
:10BC38000000000042616C6C6F632073756363657C
:10BC480065646564000000002F6D6E742F776F7255
:10BC58006B73706163652F776F726B737061636567
:10BC68002F4743432D31302D706970656C696E65BF
:10BC78002F6A656E6B696E732D4743432D31302DE6
:10BC8800706970656C696E652D3333385F32303298
:10BC980031313031385F3136333435313632303343
:10BCA8002F7372632F6E65776C69622F6E65776C80
:10BCB80069622F6C6962632F7374646C69622F64A4
:10BCC800746F612E630000002F6D6E742F776F7292
:10BCD8006B73706163652F776F726B7370616365E7
:10BCE8002F4743432D31302D706970656C696E653F
:10BCF8002F6A656E6B696E732D4743432D31302D66
:10BD0800706970656C696E652D3333385F32303217
:10BD180031313031385F31363334353136323033C2
:10BD28002F7372632F6E65776C69622F6E65776CFF
:10BD380069622F6C6962632F7374646C69622F6D1A
:10BD4800707265632E6300000080E03779C3414359
:10BD5800176E05B5B5B89346F5F93FE9034F384D69
:10BD6800321D30F94877825A3CBF737FDD4F157515
:10BD7800000000000000F03F000000000000244028
:10BD880000000000000059400000000000408F4003
:10BD9800000000000088C34000000000006AF8406E
:10BDA8000000000080842E4100000000D012634192
:10BDB8000000000084D797410000000065CDCD4108
:10BDC800000000205FA00242000000E876483742E9
:10BDD800000000A2941A6D42000040E59C30A24287
:10BDE8000000901EC4BCD64200003426F56B0C43FC
:10BDF8000080E03779C3414300A0D88557347643A3
:10BE080000C84E676DC1AB43003D9160E458E14303
:10BE1800408CB5781DAF154450EFE2D6E41A4B4478
:10BE280092D54D06CFF08044F64AE1C7022DB544BD
:10BE3800B49DD9794378EA44050000001900000050
:10BE48007D000000202020202020202020202020ED
:10BE5800202020203030303030303030303030301A
:10BE6800303030302C2066756E6374696F6E3A20FE
:10BE780000000000617373657274696F6E2022257B
:10BE88007322206661696C65643A2066696C652076
:10BE9800222573222C206C696E6520256425732564
:10BEA800730A000043000000504F53495800000037
:10BEB8002E000000002020202020202020202828DC
:10BEC8002828282020202020202020202020202052
:10BED8002020202020881010101010101010101092
:10BEE80010101010100404040404040404040410C2
:10BEF8001010101010104141414141410101010150
:10BF08000101010101010101010101010101010119
:10BF18001010101010104242424242420202020225
:10BF280002020202020202020202020202020202E9
:10BF38001010101020000000000000000000000099
:10BF480000000000000000000000000000000000E9
:10BF580000000000000000000000000000000000D9
:10BF680000000000000000000000000000000000C9
:10BF780000000000000000000000000000000000B9
:10BF880000000000000000000000000000000000A9
:10BF98000000000000000000000000000000000099
:10BFA8000000000000000000000000000000000089
:08BFB800000000000000000081
:08BFC0006C48FF7F0100000046
:08BFC80041790008E5020008C0
:04BFD000C1020008A2
:10BFD4000090D0030090D003010000001000000086
:10BFE40018000024000000000000000004030024E6
:10BFF4006C030024D40300240000000000000000AF
:10C00400000000000000000000000000000000002C
:10C01400000000000000000000000000000000001C
:10C02400000000000000000000000000000000000C
:10C0340000000000000000000000000000000000FC
:10C0440000000000000000000000000000000000EC
:10C0540000000000000000000000000000000000DC
:10C0640000000000000000000000000000000000CC
:10C0740000000000000000000000000000000000BC
:10C0840000000000000000000000000000000000AC
:10C0940001000000000000000E33CDAB34126DE649
:10C0A400ECDE05000B0000000000000000000000B2
:10C0B400000000000000000000000000000000007C
:10C0C400000000000000000000000000000000006C
:10C0D400000000000000000000000000000000005C
:10C0E400000000000000000000000000000000004C
:10C41400D00A0024000000000000000044040024AE
:10C42400440400244C0400244C0400245404002438
:10C43400540400245C0400245C04002464040024E8
:10C44400640400246C0400246C0400247404002498
:10C45400740400247C0400247C0400248404002448
:10C46400840400248C0400248C04002494040024F8
:10C47400940400249C0400249C040024A4040024A8
:10C48400A4040024AC040024AC040024B404002458
:10C49400B4040024BC040024BC040024C404002408
:10C4A400C4040024CC040024CC040024D4040024B8
:10C4B400D4040024DC040024DC040024E404002468
:10C4C400E4040024EC040024EC040024F404002418
:10C4D400F4040024FC040024FC04002404050024C7
:10C4E400040500240C0500240C0500241405002474
:10C4F400140500241C0500241C0500242405002424
:10C50400240500242C0500242C05002434050024D3
:10C51400340500243C0500243C0500244405002483
:10C52400440500244C0500244C0500245405002433
:10C53400540500245C0500245C05002464050024E3
:10C54400640500246C0500246C0500247405002493
:10C55400740500247C0500247C0500248405002443
:10C56400840500248C0500248C05002494050024F3
:10C57400940500249C0500249C050024A4050024A3
:10C58400A4050024AC050024AC050024B405002453
:10C59400B4050024BC050024BC050024C405002403
:10C5A400C4050024CC050024CC050024D4050024B3
:10C5B400D4050024DC050024DC050024E405002463
:10C5C400E4050024EC050024EC050024F405002413
:10C5D400F4050024FC050024FC05002404060024C2
:10C5E400040600240C0600240C060024140600246F
:10C5F400140600241C0600241C060024240600241F
:10C60400240600242C0600242C06002434060024CE
:10C61400340600243C0600243C060024440600247E
:10C62400440600244C0600244C060024540600242E
:10C63400540600245C0600245C06002464060024DE
:10C64400640600246C0600246C060024740600248E
:10C65400740600247C0600247C060024840600243E
:10C66400840600248C0600248C06002494060024EE
:10C67400940600249C0600249C060024A40600249E
:10C68400A4060024AC060024AC060024B40600244E
:10C69400B4060024BC060024BC060024C4060024FE
:10C6A400C4060024CC060024CC060024D4060024AE
:10C6B400D4060024DC060024DC060024E40600245E
:10C6C400E4060024EC060024EC060024F40600240E
:10C6D400F4060024FC060024FC06002404070024BD
:10C6E400040700240C0700240C070024140700246A
:10C6F400140700241C0700241C070024240700241A
:10C70400240700242C0700242C07002434070024C9
:10C71400340700243C0700243C0700244407002479
:10C72400440700244C0700244C0700245407002429
:10C73400540700245C0700245C07002464070024D9
:10C74400640700246C0700246C0700247407002489
:10C75400740700247C0700247C0700248407002439
:10C76400840700248C0700248C07002494070024E9
:10C77400940700249C0700249C070024A407002499
:10C78400A4070024AC070024AC070024B407002449
:10C79400B4070024BC070024BC070024C4070024F9
:10C7A400C4070024CC070024CC070024D4070024A9
:10C7B400D4070024DC070024DC070024E407002459
:10C7C400E4070024EC070024EC070024F407002409
:10C7D400F4070024FC070024FC07002404080024B8
:10C7E400040800240C0800240C0800241408002465
:10C7F400140800241C0800241C0800242408002415
:10C80400240800242C0800242C08002434080024C4
:10C81400340800243C0800243C080024FFFFFFFFE8
:10C8240000000200430000000000000000000000BF
:10C8340000000000000000000000000000000000F4
:10C8440000000000430000000000000000000000A1
:10C8540000000000000000000000000000000000D4
:10C864000000000043000000000000000000000081
:10C8740000000000000000000000000000000000B4
:10C884000000000043000000000000000000000061
:10C894000000000000000000000000000000000094
:10C8A4000000000043000000000000000000000041
:10C8B4000000000000000000000000000000000074
:10C8C4000000000043000000000000000000000021
:10C8D4000000000000000000000000000000000054
:10C8E4000000000043000000000000000000000001
:10C8F4000000000000000000000000000000000034
:10C904000000000099BA000885B400080000000087
:10C91400BCBE0008B8BE000874BB000874BB0008A5
:10C9240074BB000874BB000874BB000874BB000827
:10C9340074BB000874BB000874BB0008FFFFFFFF52
:10C94400FFFFFFFFFFFFFFFFFFFF00000100415358
:10C9540043494900000000000000000000000000FE
:10C96400000000000000000000000000000041532F
:10C9740043494900000000000000000000000000DE
:10C9840000000000000000000000000000000000A3
:0400000508001E05CC
:00000001FF
